:020000040800F2
:10000000800F0020A52A0008A5040008A704000806
:10001000AB040008AF040008B304000800000000AF
:10002000000000000000000000000000B70400080D
:10003000B904000800000000BB040008BD0400086B
:10004000BF2A0008BF2A0008BF2A0008BF2A0008EC
:10005000BF2A0008BF2A0008BF2A0008BF2A0008DC
:10006000BF2A0008BF2A0008BF2A0008BF2A0008CC
:10007000BF2A0008BF2A0008BF2A0008BF2A0008BC
:10008000BF2A0008BF2A0008BF2A0008BF2A0008AC
:10009000BF040008BF2A0008BF2A0008BF2A0008C2
:1000A000BF2A0008BF2A0008BF2A0008BF2A00088C
:1000B000BF2A0008E3550008BF2A0008BF2A00082D
:1000C000BF2A0008BF2A0008BF2A0008BF2A00086C
:1000D000BF2A000803510008D7040008D90400080B
:1000E000BF2A0008BF2A0008C704000800F002F871
:1000F00000F06DF80AA090E8000C82448344AAF155
:100100000107DA4501D100F062F8AFF2090EBAE852
:100110000F0013F0010F18BFFB1A43F0010318473B
:10012000C4A30000E4A300000A444FF0000C10F840
:10013000013B13F0070408BF10F8014B1D1108BF65
:1001400010F8015B641E05D010F8016B641E01F805
:10015000016BF9D113F0080F1EBF10F8014BAD1C55
:100160000C1B09D16D1E58BF01F801CBFAD505E073
:1001700014F8016B01F8016B6D1EF9D59142D6D3CD
:10018000704700000023002400250026103A28BFF5
:1001900078C1FBD8520728BF30C148BF0B607047F9
:1001A000662909F01C87642907F02682782907F060
:1001B0005F82002070471FB507F0B0FD04000020EB
:1001C000002108F0BDFEE0601FBD10B510BD07F0B6
:1001D000C1FE1146FFF7EFFF00F008F807F0DFFE61
:1001E00003B4FFF7F2FF03BC04F03CFF00F044F857
:1001F0004FF4E13004F044FF04F07FFE04F0B2FE5F
:1002000000F09FF800F047F803F014FAC82005F05A
:1002100083F807F0F6F81449087005F050FA6420E6
:1002200005F07AF805F064FD41F61F41092005F05C
:1002300087FE17E005F05FF90B48007801280CD025
:1002400004F0B1FA4FF4FA7005F066F804F0A5FA7C
:100250004FF4FA7005F060F804E004F0A4FA01200D
:1002600005F05AF8E6E700000000002010B5012173
:10027000084601F02BF810BD10B505F08EFEFFF713
:10028000F5FF0121080701F02EF805F027F804F02A
:1002900081FF10BD704710B5002000F077FF0121ED
:1002A000C80501F020F810BD03207849086000203F
:1002B00077490870704777480121754A1170817A33
:1002C00019B10521714A116002E001216F4A1160E4
:1002D000704710B5012000F010FF00BF212000F092
:1002E000CAFE0028FAD0002000F019FF002000F01C
:1002F00013FF002000F09CFE30BF10BD10B500F0D1
:10030000D6FE654908704FF4803000F091FE00BFC2
:10031000312000F0B0FE0028FAD0012000F0FCFEF1
:1003200000BF392000F0A7FE0028FAD0022000F01C
:10033000F6FE00BF00F0FCFE0828FBD110BD7047A0
:1003400070470EB54FF4802000F0BDF94FF48020C7
:10035000019008208DF8090000208DF80800012088
:100360008DF80A0001A800F037F94FF4A06000F002
:10037000B7F814208DF8000002208DF8010000204D
:100380008DF8020001208DF80300684600F0ADF8FA
:100390002A208DF8000001208DF80100684600F049
:1003A000A4F80EBD70477047F0B5044616460BB171
:1003B000022500E001252A4600201FE004F01F0569
:1003C0000A2D08DA05F1300707F0FF0C00FB02F7F1
:1003D00001F807C007E005F1370707F0FF0C00FB45
:1003E00002F701F807C033B14FF0000C00FB02F731
:1003F0007F1C01F807C06409451CE8B2B042DDDB90
:10040000F0BD00212548008808B10120704719B1CE
:10041000224801800120F9E70020F7E710B5FFF737
:10042000F0FF1E480088022802DA02201B490880DB
:1004300010BD10B50446FFF7F1FF10BD2DE9F047E0
:1004400004468A464FF0AA373D461548D0F800804A
:10045000001DD0F80090001D066806F4404086EAB2
:10046000900789EA080505F4404085EA90050023D5
:10047000062221463846FFF797FF00230622A11DDA
:100480002846FFF791FFBDE8F087000040010020FB
:1004900006000020000200200200002004000020CE
:1004A000E8F7FF1F704700BFFEE700BFFEE700BF91
:1004B000FEE700BFFEE7704770477047704710B512
:1004C00003F0EEFE10BD10B5012004490870800451
:1004D00000F0F9F810BD70477047000006000020DA
:1004E00031490143314A1160704770B50021002342
:1004F0000F22C47804B32D4C246804F4E064C4F5DE
:10050000E064210AC1F10403CA40447804FA03F10B
:100510008478144021430901254C0678A1550478BC
:1005200004F01F050124AC4005786D11AD0005F104
:10053000E025C5F8004109E0047804F01F05012416
:10054000AC401C4D0678761145F8264070BD1A4A1D
:100550000A400243154B1B1F1A60704739B1134AFA
:10056000121D12680243114B1B1D1A6006E00F4A50
:10057000121D126882430D4B1B1D1A607047042820
:1005800008D14FF0E021096941F004014FF0E02269
:10059000116107E04FF0E021096921F004014FF0FB
:1005A000E0221161704700000000FA050CED00E048
:1005B00000E400E080E100E080FFFF1F00204449EC
:1005C0000860091D0860091D0860091D0860414890
:1005D0003F4914310860704700213D498279002A63
:1005E0003AD00A46126803689A430B461A600A1DFD
:1005F000126803689A430B1D1A60027911440A6855
:1006000003681A430A60324A0832126803689A4340
:100610002F4B08331A601A1D126803689A432C4B3B
:100620000C331A604279102A0ED11A1F126803681F
:100630001A43274B08331A601A1D126803681A43BD
:10064000234B0C331A600DE02149427911440A68AA
:1006500003681A430A6005E0027911440A680368D6
:100660009A430A6070470021016001710C214171B9
:100670000021817170471649103109680143144AFD
:1006800010321160704701460020114A143212687E
:100690000A400AB1012000E0002070470C491431E3
:1006A00008607047014600200022094B1B6803EADE
:1006B0000102074B14331B680B4013B10AB1012030
:1006C00000E00020704702491431086070470000C4
:1006D00000040140FFFF0F0001460020FE4A1068A1
:1006E00000F03800084310607047FB49096821F0AA
:1006F0000801F94A11601146096801431160704709
:10070000F549096821F01001F34A116011460968A2
:10071000014311607047F148EF494860F048486074
:100720007047EE48EC494860ED4848607047EA4839
:10073000006940F08000E84908617047E6480069B8
:1007400040F08000E449086170470420E249C9682C
:1007500001F0010109B101200EE0DF49C96801F093
:10076000040109B1022007E0DB49C96801F010016A
:1007700009B1032000E00420704700B502460423BD
:10078000FFF7E3FF034603E0FFF7DFFF0346521ED8
:10079000012B01D1002AF7D102B90523184600BD6B
:1007A00030B5044604254FF43020FFF7E6FF054638
:1007B000042D17D1C848006940F00200C6490861FD
:1007C00008464461006940F0400008614FF4302061
:1007D000FFF7D3FF0546C048006941F6FD710840A8
:1007E000BD490861284630BD10B504244FF43020BF
:1007F000FFF7C3FF0446042C16D1B748006940F048
:100800000400B54908610846006940F040000861ED
:100810004FF43020FFF7B1FF0446AF48006941F6BE
:10082000FB710840AC490861204610BD00B5024686
:100830000423FFF78AFF034603E0FFF786FF034622
:10084000521E012B01D1002AF7D102B90523184607
:1008500000BD10B504244FF43020FFF7E7FF044635
:10086000042C16D19C48006940F004009A490861A4
:100870000846006940F0400008614FF43020FFF75F
:10088000D5FF04469448006941F6FB71084092493F
:100890000861204610BD00208F49C96901F002019E
:1008A00009B1012000E00020704730B5A5250424DF
:1008B000FFF7F1FF00B100254FF43020FFF75DFF97
:1008C0000446042C3AD1854883498860844888606E
:1008D0000846006940F0200008610846006940F0C1
:1008E000400008614FF43020FFF747FF0446042C16
:1008F0001BD17948006941F6DF71084076490861EB
:100900000846006940F01000086176480580E00262
:10091000FFF733FF0446052C10D06F48006941F6FD
:10092000EF7108406C49086108E0052C06D06A4860
:10093000006941F6EF71084067490861204630BD03
:1009400078B506460C46042500200090E802FFF723
:1009500014FF0546042D24D15F48006940F00100D2
:100960005D4908613480E802FFF707FF0546042D62
:1009700010D1B01C0090200C00990880E802FFF70D
:10098000FCFE05465448006941F6FE710840524994
:10099000086106E05048006941F6FE7108404E4982
:1009A0000861284678BD70B504460D460426F0025D
:1009B000FFF7E3FE0646042E11D14748006940F0D8
:1009C0000100454908612580F002FFF7D6FE064682
:1009D0004148006941F6FE7108403F4908613046D0
:1009E00070BD70B505460E460424E002FFF7C5FE53
:1009F0000446042C17D13948374988603848886044
:100A00000846006940F0100008612E80E002FFF700
:100A1000B4FE0446052C06D02F48006941F6EF715C
:100A200008402D490861204670BD2DE9F043044679
:100A30004FF6FF763746B046B1460425E443E6B2AA
:100A4000C4F30727C4F307484FEA1469E802FFF725
:100A500094FE0546042D49D120481F49886020484E
:100A600088600846006940F010000861FF2E06D03B
:100A70001C4808300680E802FFF77FFE0546042D7B
:100A800008D1FF2F06D017480A300780E802FFF789
:100A900074FE0546042D0AD1B8F1FF0F07D01148A6
:100AA0000C30A0F80080E802FFF767FE0546042D31
:100AB0000AD1B9F1FF0F07D00A480E30A0F8009014
:100AC000E802FFF75AFE0546052D0FD002480069DF
:100AD00041F6EF71084007E000200240230167451E
:100AE000AB89EFCD00F8FF1F664908612846BDE8D5
:100AF000F08330B5054604244FF43020FFF73DFE67
:100B00000446042C41D160485E4988605F48886093
:100B10000846006940F0200008610846006940F07E
:100B2000400008614FF43020FFF727FE0446042CF4
:100B300022D15448006941F6DF71084051490861EB
:100B40000846006940F0100008611DB100205049BE
:100B5000088002E0A5204E4908804FF43020FFF7BE
:100B60000CFE0446052C10D04648006941F6EF7192
:100B700008404449086108E0052C06D04148006956
:100B800041F6DF7108403F490861204630BDF0B5AD
:100B900005460E46174604243B483A4988603B48C0
:100BA0008860E002FFF7E9FD0446042C19D13548BE
:100BB000006940F010003349086147F0F800304305
:100BC00028433349891C0880E002FFF7D6FD04461C
:100BD000052C06D02B48006941F6EF7108402949E1
:100BE00008612046F0BD2748C06980087047254845
:100BF000006A704700202349096801F0200109B10B
:100C0000012000E00020704729B11E4A126902430A
:100C10001C4B1A6104E01B4A12698243194B1A618A
:100C2000704701460020012908D1164AD26902F016
:100C300001020AB1012008E0002006E0114AD26852
:100C40000A400AB1012000E0002070470D49C86049
:100C5000704704200B49C96801F0010109B1012066
:100C60000EE00849C96801F0040109B1022007E05B
:100C70000449C96801F0100109B1032000E0042013
:100C8000704700000020024023016745AB89EFCD8B
:100C900000F8FF1F10B50446CC48844208D101215A
:100CA000042000F02DFB0021042000F029FB46E089
:100CB000C748844208D10121082000F021FB00210F
:100CC000082000F01DFB3AE0C248844208D101210F
:100CD000102000F015FB0021102000F011FB2EE089
:100CE000BD48844208D10121202000F009FB0021E9
:100CF000202000F005FB22E0B848844208D1012101
:100D0000402000F0FDFA0021402000F0F9FA16E042
:100D1000B348844208D10121802000F0F1FA00217B
:100D2000802000F0EDFA0AE0AE48844207D10121AC
:100D3000801500F0E5FA0021A01500F0E1FA10BDE1
:100D400010B50121084600F0DBFA0021012000F077
:100D5000D7FA10BD2DE9F0410246002500260020FB
:100D600000230024002791F803C00CF00F0591F830
:100D700003C00CF0100CBCF1000F03D091F802C0BE
:100D80004CEA050591F800C0BCF1000F31D01468A1
:100D900000202BE04FF0010C0CFA00F3B1F800C07A
:100DA0000CEA03069E4220D183004FF00F0C0CFA90
:100DB00003F7BC4305FA03FC4CEA040491F803C0B2
:100DC000BCF1280F06D14FF0010C0CFA00FCC2F860
:100DD00014C00AE091F803C0BCF1480F05D14FF0F0
:100DE000010C0CFA00FCC2F810C0401C0828D1D33A
:100DF0001460B1F800C0BCF1FF0F34DD546800206E
:100E00002EE000F1080C4FF0010808FA0CF3B1F8DD
:100E100000C00CEA03069E4221D183004FF00F0C64
:100E20000CFA03F7BC4305FA03FC4CEA040491F8FE
:100E300003C0BCF1280F05D100F1080C08FA0CF82A
:100E4000C2F8148091F803C0BCF1480F07D100F13B
:100E5000080C4FF0010808FA0CF8C2F81080401C8A
:100E60000828CED35460BDE8F0814FF6FF710180B1
:100E7000022181700421C1707047024600209368EE
:100E80000B400BB1012000E000207047014688684C
:100E900080B2704702460020D3680B400BB101209E
:100EA00000E0002070470146C86880B270470161C9
:100EB0007047416170470AB1016100E041617047CC
:100EC000C16070474FF480320A4382618161826160
:100ED00082698269704702460020434B18684FF6CA
:100EE0008073184040EA021008433F4B1860704777
:100EF0003E49C8617047F0B50A460023002400212E
:100F0000002500F00046B6F1004F02D1364EF169DF
:100F100001E0354E7168C0F3034583B200F440161A
:100F2000B6F5401F08D121F070612F4E766826F08B
:100F300070662D4F7E6012E000F48016B6F5801FBB
:100F400006D1032606FA05F4A14341F0706106E0DC
:100F5000460D360103FA06F6B14341F0706122B145
:100F6000460D360103FA06F6314300F00046B6F1AD
:100F7000004F02D11C4EF16101E01B4E7160F0BDCB
:100F800030B500228B071C0F0F2303FA04F2164B17
:100F900008338C1053F824309343134C08348D10CD
:100FA00044F8253023468C1053F824308C07240F46
:100FB00000FA04F423430C4C08348D1044F8253017
:100FC00030BD0A49DC31086070470000000801406C
:100FD000000C0140001001400014014000180140C5
:100FE000001C0140002001400000014000002042A0
:100FF000DF48006840F00100DD49086008464068AD
:10100000DC490840DA49486008460068DA49084087
:10101000D74908600846006820F480200860084628
:10102000406820F4FE0048604FF41F00886070475D
:10103000CF49096821F48031CD4A11601146096811
:1010400021F480211160B0F5803F03D0B0F5802FEE
:101050000ED106E0C649096841F48031C44A1160E6
:1010600007E0C349096841F4A021C14A116000E0CA
:1010700000BF00BF704710B50146002200230020CA
:101080004A11012A02D1BA4C236806E0022A02D191
:10109000B74C236A01E0B64C636A01F01F020124D9
:1010A00094401C400CB1012000E0002010BD38B578
:1010B000002000900024002500BF3120FFF7DBFF57
:1010C00005460098401C00900098B0F5A06F01D034
:1010D000002DF2D03120FFF7CEFF08B1012400E04F
:1010E0000024204638BD01460020A14A106820F0A7
:1010F000F80040EAC10010607047A04908607047DE
:10110000024600209A4B586820F47C1042EA010302
:101110001843974B586070479849086670470146D6
:101120000020934A506820F0030008435060704745
:101130008F48406800F00C007047014600208C4A40
:10114000506820F0F00008435060704701460020CE
:10115000874A506820F4E0600843506070470146B9
:101160000020834A506820F4605040EAC10050607B
:10117000704729B17E4A527A02437D4B5A7204E08D
:101180007B4A527A82437A4B5A7270477B49D831F4
:101190000860704701460020754A506820F44040BE
:1011A0000843506070470021714A20321170704A24
:1011B00082F82010012802D004280AD104E001217D
:1011C0006B4A2032117005E00521694A2032117006
:1011D00000E000BF00BF704769490860704764497C
:1011E000096A0143624A11627047654944390860DF
:1011F000704730B500210022002400235C4D6D684B
:1012000005F00C0121B1042905D0082923D105E0FE
:101210005C4D056022E05B4D05601FE0544D6D683C
:1012200005F47012524D6D6805F48034022505EB0B
:1012300092421CB9544D554305600BE04C4D6D680E
:1012400005F400351DB1504D5543056002E04D4D8C
:101250005543056002E04B4D056000BF00BF444DA3
:101260006D6805F0F0010909484D6B5C0568DD40CB
:1012700045603F4D6D6805F4E061090A434D6B5CC4
:101280004568DD4085603A4D6D6805F46051C90AD6
:101290003E4D6B5C4568DD40C560354D6D6805F4BD
:1012A0004041890B3A4D6B5CC568B5FBF3F50561B0
:1012B00030BD29B12E4A526902432D4B5A6104E0D8
:1012C0002B4A526982432A4B5A61704729B1284AF6
:1012D00092690243264B9A6104E0254A926982434F
:1012E000234B9A61704729B1214AD2690243204BAE
:1012F000DA6104E01E4AD26982431D4BDA6170470D
:1013000029B11B4AD2680243194BDA6004E0184A3B
:10131000D2688243164BDA60704729B1144A1269C9
:101320000243134B1A6104E0114A12698243104BC5
:101330001A61704712494039086070470F49C86404
:1013400070470B49C87170470948406A40F0807087
:1013500007494862704701460020054A92680A40E2
:101360000AB1012000E000207047014988727047EF
:10137000001002400000FFF8FFFFF6FE00004242AE
:101380008004424200127A0000093D00070000205C
:101390001700002010B50446BE48844208D1012140
:1013A0008014FFF7ADFF0021A014FFF7A9FF16E09E
:1013B000B948844208D101210014FFF7AEFF002193
:1013C0002014FFF7AAFF0AE0B448844207D10121A4
:1013D000C013FFF7A2FF0021E013FFF79EFF10BD2F
:1013E00010B50022028802F441520B884C88234336
:1013F0008C882343CC8823430C8923434C89234383
:101400008C892343CC8923431A430280838B4FF278
:10141000FF74234083830B8A038210BD2DE9F04FB4
:1014200085B005460C464FF0000902274FF0000832
:101430004FF0010B0026B246A88B4FF24001084046
:10144000A88302202884B5F81C90A068022801D146
:1014500000BF38E0A08810B94FF0010B01E04FF059
:10146000020B8D48854200D100E000BF6846FFF7BF
:10147000C0FEDDF800A0E088B0F5007F0AD14FEA99
:101480001A2000EB80004000A168B0FBF1F0401D85
:1014900086B20BE04FEA4B10BAFBF0F000EB800095
:1014A0004000A168B0FBF1F0401D86B20A20B6FBF7
:1014B000F0F606F00108A6EB0800C0F34F074FF660
:1014C000FF7000EA0828022F01DBFF2F02DD022750
:1014D0004FF00008E08840EA080038432884A088DC
:1014E000A1890843618808432188084340F40060CB
:1014F00040EA0909A5F81C9005B0BDE8F08F00216D
:10150000018041808180C180018141818181C181CF
:101510000721018270470021018041808180C180C4
:101520000221816000218181704721B1028842F04F
:101530004002028004E002884FF6BF731A40028026
:10154000704721B1828B42F48062828304E0828BF7
:101550004FF6FF331A408283704730B500240023D2
:101560000C110125A540ABB21AB185881D438580B9
:1015700002E085889D43858030BD1AB183880B4386
:10158000838002E083888B4383807047818170472A
:101590000146888970474FF6FF62914204D0028865
:1015A00042F48072028004E002884FF6FF631A4022
:1015B0000280704721B1828842F00402828004E0F8
:1015C00082884FF6FB731A408280704702884FF280
:1015D000FF731A40028002880A4302807047018824
:1015E00041F480510180704721B1028842F40052D9
:1015F000028004E002884DF6FF731A4002807047B3
:1016000002460020012901D0108B00E0908A70472B
:101610000146088A7047B1F5804F04D1028842F430
:101620008042028004E002884BF6FF731A40028079
:1016300070470246002013890B400BB1012000E0E7
:1016400000207047CA4302817047F0B5024600206F
:1016500000240023002501F00F070126BE40B4B28C
:101660000B1101269E40B3B2968806EA030516893F
:10167000264016B10DB1012000E00020F0BD10B5EC
:10168000002201F00F040123A3409AB2D343038147
:1016900010BD00000030014000380040003C004018
:1016A00010B50446FE48844208D10121C014FFF75A
:1016B00027FE0021E014FFF723FEC4E0B4F1804FC1
:1016C00008D101210846FFF728FE00210120FFF77D
:1016D00024FEB8E0F348844208D101210220FFF73C
:1016E0001CFE00210220FFF718FEACE0EE48844209
:1016F00008D101210420FFF710FE00210420FFF78C
:101700000CFEA0E0E948844208D101210820FFF73F
:1017100004FE00210820FFF700FE94E0E448844224
:1017200008D101211020FFF7F8FD00211020FFF75C
:10173000F4FD88E0DF48844208D101212020FFF732
:10174000ECFD00212020FFF7E8FD7CE0DA48844230
:1017500008D101214014FFF7D3FD00216014FFF7E9
:10176000CFFD70E0D548844209D10121C804FFF7BC
:10177000C7FD00214FF40020FFF7C2FD63E0D04811
:10178000844209D101210805FFF7BAFD00214FF479
:101790008010FFF7B5FD56E0CA48844209D1012107
:1017A0004805FFF7ADFD00214FF40010FFF7A8FD3D
:1017B00049E0C548844208D101214020FFF7ADFD32
:1017C00000214020FFF7A9FD3DE0C048844208D138
:1017D00001218020FFF7A1FD00218020FFF79DFD62
:1017E00031E0BB48844208D101218015FFF795FD07
:1017F0000021A015FFF791FD25E0B648844209D1EC
:1018000001210804FFF77CFD00214FF48030FFF731
:1018100077FD18E0B048844209D101214804FFF760
:101820006FFD00214FF40030FFF76AFD0BE0AB487D
:10183000844208D101218804FFF762FD00214FF4A2
:101840008020FFF75DFD10BD00220288944B984276
:101850000ED0994B98420BD0B0F1804F08D0914BED
:10186000984205D0904B984202D0904B984204D1B8
:101870004FF68F731A404B881A438D4B984207D00E
:101880008C4B984204D04FF6FF431A40CB881A4342
:1018900002808B8883850B880385814B98420BD00F
:1018A000854B984208D08B4B984205D08A4B984282
:1018B00002D08A4B984201D10B7A0386012383829E
:1018C000704770B5002400220023058C4FF6FE7689
:1018D00035400584028C8388048B4FF68F752C402D
:1018E000B51E2C400D882C43751E2A400D892A43B5
:1018F0004D882A436A4DA8420BD06F4DA84208D0AC
:10190000744DA84205D0744DA84202D0734DA84230
:1019100013D14FF6F7752A404D892A434FF6FB75D0
:101920002A408D882A434FF6FF652B404FF6FF551E
:101930002B408D892B43CD892B4383800483CD8815
:101940008586028470BD70B5002400220023058CBA
:101950004FF6EF7635400584028C8388048B48F679
:10196000FF752C404FF6FF452C400D884FF6FF7653
:1019700006EA05252C434FF6DF752A400D8906EA55
:1019800005152A434D8806EA05152A43444DA84209
:1019900002D0494DA8421DD14FF67F752A404D898E
:1019A0004FF6FF7606EA05152A434FF6BF752A4023
:1019B0008D8806EA05152A434FF6FF352B404FF276
:1019C000FF752B408D8906EA85052B43CD8906EAF4
:1019D00085052B4383800483CD880587028470BDF1
:1019E00070B5002400220023058C4FF6FF663540B9
:1019F0000584028C8388848B4FF68F752C404FF6BC
:101A0000FC752C400D882C434FF6FF552A400D895C
:101A10004FF6FF7606EA05252A434D8806EA052596
:101A20002A431F4DA84202D0234DA8421DD14FF298
:101A3000FF752A404D894FF6FF7606EA05252A43B1
:101A40004FF6FF352A408D8806EA05252A434EF6D3
:101A5000FF752B404DF6FF752B408D8906EA051565
:101A60002B43CD8906EA05152B4383808483CD88DB
:101A70008587028470BD70B5002200230024058C88
:101A80004EF6FF7635400584038C8488828B48F6B9
:101A9000FF752A404FF6FF452A400D8820E00000E0
:101AA000002C01400004004000080040000C0040F1
:101AB000001000400014004000340140004C014080
:101AC000005001400054014000180040001C00403C
:101AD0000020004000400140004401400048014017
:101AE0004FF6FF7606EA05252A434DF6FF752B4093
:101AF0000D8906EA05352B434D8806EA05352B434B
:101B0000FA4DA84202D0FA4DA84208D14BF6FF7513
:101B10002C408D894FF6FF7606EA85152C4384808C
:101B20008283CD88A0F84050038470BD828B4FF231
:101B3000FF331A408283828B4FF6FF7303EA01233F
:101B40001A4382837047F0B50C46154600220021E7
:101B50000026078C4EF6FF7C07EA0C070784828B71
:101B6000018C4FF6FF7707EA043640F6FF473A400C
:101B70004FF6FF7707EA05273A434FF6FF7707EA64
:101B800003373A43D94FB8420ED0D94FB8420BD0A1
:101B9000B0F1804F08D0D74FB84205D0D64FB842E9
:101BA00002D0D64FB84206D14DF6FF77394046F401
:101BB0008057394305E047F6FF57394044F48057D2
:101BC000394382830184F0BD828B4FF6F3731A4050
:101BD0008283828B0A4382837047F0B50C46154698
:101BE000002200210026078C4FF6FF6C07EA0C0745
:101BF0000784828B018C4FF6FF7707EA04264FF6A5
:101C00000C773A404FF6FF7707EA03172F433A4322
:101C1000B64FB8420ED0B64FB8420BD0B0F1804F9D
:101C200008D0B44FB84205D0B34FB84202D0B34F3A
:101C3000B84206D14FF6FF57394046F48077394312
:101C400005E04FF2FF57394044F4807739438283EF
:101C50000184F0BD028B4FF2FF331A400283028BE6
:101C60004FF6FF7303EA01231A4302837047F0B56E
:101C70000C461546002200210026078C4FF6EF7C0B
:101C800007EA0C070784028B018C4FF6FF7707EAFF
:101C9000041640F6FF473A404FF6FF7707EA03374E
:101CA0003A434FF6FF7707EA05273A438F4FB8428A
:101CB0000ED08F4FB8420BD0B0F1804F08D08D4F6F
:101CC000B84205D08C4FB84202D08C4FB84206D1F2
:101CD0004FF6DF77394046F01007394305E04FF6FD
:101CE0005F77394044F01007394302830184F0BD27
:101CF000028B4FF6F3731A400283028B0A4302836E
:101D00007047F0B50C46154600220021068C4FF6B0
:101D1000FE773E400684028B018C4FF60C763240F3
:101D20007E1C06EA03162E433243704EB0420ED09C
:101D30006F4EB0420BD0B0F1804F08D06D4EB04224
:101D400005D06D4EB04202D06C4EB04206D14FF677
:101D5000FD76314044F00106314305E04FF6F5765B
:101D6000314044F00106314302830184F0BD70B577
:101D700005460C465D4885420ED05D4885420BD035
:101D8000B5F1804F08D05B48854205D05A4885425E
:101D900002D05A48854200D100E000BF208850B9E7
:101DA0002389A28861882846FFF7ABFFE18828468F
:101DB000FFF79EFF25E0208804280AD12389A28806
:101DC00061882846FFF753FFE1882846FFF742FF66
:101DD00017E0208808280AD12389A288618828462C
:101DE000FFF7FBFEE1882846FFF7EEFE09E02389B6
:101DF000A28861882846FFF7A6FEE1882846FFF7FB
:101E000095FE70BD2DE9F04105460C4600260127E0
:101E1000608808B9022600E00026A088012801D1C8
:101E2000022700E001272088A0B92389A2886188C1
:101E30002846FFF766FFE1882846FFF759FF238908
:101E40003A4631462846FFF712FFE1882846FFF759
:101E500001FF13E02389A28861882846FFF707FF66
:101E6000E1882846FFF7F6FE23893A4631462846A0
:101E7000FFF747FFE1882846FFF73AFFBDE8F0810A
:101E80000A884B881A438B881A43CB881A430B89DC
:101E90001A434B891A438B891A43A0F84420704790
:101EA0004FF6FF71818000210180C1804180017265
:101EB00070470021018041808180C1800181418182
:101EC0008181C18170470021018041800121818091
:101ED0000021C18001817047002101804180818003
:101EE000C18001814181818170470000002C014047
:101EF000003401400004004000080040000C004095
:101F000021B1028842F00102028004E002884FF60B
:101F1000FE731A400280704731B1B0F8442042F499
:101F20000042A0F8442005E0B0F84420C2F30E02BD
:101F3000A0F8442070471AB183890B43838102E0E3
:101F400083898B43838170478182704741EA020312
:101F5000A0F8483070471AB183890B43838102E0AF
:101F600083898B438381704701894FF6F872114052
:101F7000018170470A46002101894FF68F7319408D
:101F800011430181704730B504460D46294620466D
:101F9000FFF7F0FF208940F00700208130BD2DE9D8
:101FA000F04104460D4616461F46602D06D13B46BD
:101FB000012231462046FFF75AFE05E03B4601224A
:101FC00031462046FFF79DFE29462046FFF7D2FF07
:101FD000208940F007002081BDE8F08130B50C4633
:101FE00000210189C9B24FF6FF7505EA03251543A3
:101FF00025432943018130BD2DE9F04105460E46B8
:1020000017469846002443463A4631462846FFF78D
:10201000E5FF2C894FF6F870044044F007044FF6B2
:102020008F70044044F070042C81BDE8F081F0B55D
:1020300004460D4616461F463B4632462946204674
:10204000FFF7CCFF208940F480402081F0BD01855E
:10205000828270470A46002101884FF68F7319402B
:10206000114301807047F0B50C4615461E4600210D
:10207000002200230189028B038C4FF6F877394048
:1020800021434FF6FC473A4040F201173A434FF6DE
:10209000DD773B404FF6FF7707EA06172F433B43B8
:1020A000018102830384F0BD0A460021018B4FF6B3
:1020B0008F7319401143018370470A460021018B39
:1020C00048F6FF7319404FF6FF7303EA02231943E2
:1020D000018370470A460021818B4FF68F731940A8
:1020E0001143818370470A460021818B48F6FF73B4
:1020F00019404FF6FF7303EA0223194381837047A7
:1021000021B1028842F08002028004E002884FF68A
:102110007F731A400280704721B1828842F0040226
:10212000828004E082884FF6FB731A4082807047F9
:1021300021B1828842F00802828004E082884FF652
:10214000F7731A408280704721B1828842F0010201
:10215000828004E082884FF6FE731A4082807047C6
:102160000A460021018B4FF6F77319401143018392
:1021700070470A460021018B4FF2FF7319404FF65A
:10218000FF7303EA02231943018370470A460021C3
:10219000818B4FF6F77319401143818370470A46CC
:1021A0000021818B4FF2FF7319404FF6FF7303EA52
:1021B00002231943818370470A460021018B4FF6A1
:1021C000FB7319401143018370470A460021018BBC
:1021D0004FF6FF3319404FF6FF7303EA022319430A
:1021E000018370470A460021818B4FF6FB7319402B
:1021F0001143818370470A460021818B4FF6FF33DC
:1022000019404FF6FF7303EA022319438183704795
:102210000A460021018B4FF67F7319401143018359
:1022200070470A460021018BC1F30E014FF6FF7380
:1022300003EA02231943018370470A460021818B78
:102240004FF67F7319401143818370470A4600217E
:10225000818BC1F30E014FF6FF7303EA022319438A
:10226000818370470A460021018C4FF6FD731940A7
:102270001143018470470A460021018C4FF6F77321
:1022800019401143018470470A460021018C4FF622
:10229000DF7319404FF6FF7303EA021319430184F9
:1022A00070470A460021018C4FF67F7319404FF6A4
:1022B000FF7303EA02131943018470470A460021A1
:1022C000018C4FF6FF5319404FF6FF7303EA0223C8
:1022D0001943018470470A460021018C4FF2FF73B5
:1022E00019404FF6FF7303EA022319430184704734
:1022F0000A460021018C4DF6FF7319404FF6FF731B
:1023000003EA023319430184704730B500230124E6
:102310008C40A3B2048C9C430484048C02FA01F523
:10232000ADB22C43048430BD30B5002304248C406E
:10233000A3B2048C9C430484048C02FA01F5ADB270
:102340002C43048430BD70B5034600200024184699
:10235000183001258D40ACB21D8CA5431D8409B1F8
:10236000082909D100EB6100056825F070050560BA
:102370000568154305600EE00D1FC5F34E052844A2
:10238000056825F4E045056005684FF6FF7606EA26
:1023900002263543056070BD21B1028842F0020279
:1023A000028004E002884FF6FD731A4002807047F5
:1023B00021B1028842F00402028004E002884FF654
:1023C000FB731A400280704721B1828842F080027C
:1023D000828004E082884FF67F731A4082807047C3
:1023E00002884FF6F7731A40028002880A4302807F
:1023F000704782884FF68F731A40828082880A4322
:102400008280704702894FF6F8731A400281028970
:102410000A430281704702894FF67F731A40028196
:1024200002890A4302817047818470478185704721
:10243000818670470187704781877047A0F84010F8
:10244000704702884FF6FF431A40028002880A4311
:10245000028070470146888E70470146088F70479A
:102460000146888F70470146B1F840007047014629
:10247000888C70470146088D704702460020138AF9
:102480000B400BB1012000E000207047CA430282DC
:10249000704730B50246002000230024158A05EA63
:1024A0000103958905EA010413B10CB1012000E094
:1024B000002030BDCA4302827047000010B50446B8
:1024C000FB48844209D101218803FEF719FF00214E
:1024D0004FF48040FEF714FF32E0F648844209D101
:1024E00001214804FEF719FF00214FF40030FEF7E8
:1024F00014FF25E0F048844209D101218804FEF749
:102500000CFF00214FF48020FEF707FF18E0EB4896
:10251000844209D10121C804FEF7FFFE00214FF4D7
:102520000020FEF7FAFE0BE0E548844208D10121C5
:102530000805FEF7F2FE00214FF48010FEF7EDFED5
:1025400010BD2DE9F04786B005460E460024A24690
:1025500000BFA1460027B08900B100BF2F462C8ADA
:102560004CF6FF700440F08804432C82AC894EF690
:10257000F3100440B088318908437189084304434B
:10258000AC81AC8A4FF6FF400440B0890443AC8272
:1025900001A8FEF72EFEC648874202D1DDF810A042
:1025A00001E0DDF80CA0A88900F4004040B10AEB7E
:1025B000CA0000EB0A1031684900B0FBF1F807E0EF
:1025C0000AEBCA0000EB0A1031688900B0FBF1F891
:1025D0006420B8FBF0F004012009642101FB10899C
:1025E000A88900F4004040B1322000EBC900B0FBE4
:1025F000F1F000F00700044308E0322000EB09107E
:102600006421B0FBF1F000F00F0004432C8106B010
:10261000BDE8F0874FF41651016000218180C18030
:1026200001810C21418100218181704710B5024652
:102630000020108A4FF2FF0318400B884C88234378
:102640008C882343CC8823431843108210BD00217B
:10265000018041808180C180704721B1828942F42C
:102660000052828104E082894DF6FF731A40828114
:102670007047F0B50346002400260025002040F6F0
:102680006A17B94200D100BF1846C1F3421401F0E5
:102690001F06012707FA06F5012C01D10C3004E0D2
:1026A000022C01D1103000E014301AB107682F431A
:1026B000076002E00768AF430760F0BD1AB1838A84
:1026C0000B43838202E0838A8B4383827047028AB2
:1026D0004FF6F0731A400282028A0A430282704760
:1026E00082894FF2FF731A40828182890A43828174
:1026F000704721B1828942F00202828104E082891E
:102700004FF6FD731A4082817047028A4FF6DF73DD
:102710001A400282028A0A430282704721B1028A69
:1027200042F48042028204E0028A4BF6FF731A40B0
:1027300002827047C1F30802828070470146888890
:10274000C0F308007047818941F001018181704721
:10275000028BD2B20283028B42EA012202837047CB
:10276000028B02F47F420283028B0A43028370478A
:1027700021B1828A42F02002828204E0828A4FF6EE
:10278000DF731A408282704721B1828A42F01002C0
:10279000828204E0828A4FF6EF731A408282704789
:1027A00021B1828A42F00802828204E0828A4FF6D6
:1027B000F7731A408282704721B1828942F4004245
:1027C000828103E08289C2F30E028281704721B1C7
:1027D000828A42F40062828204E0828A4FF2FF73AE
:1027E0001A4082827047828A4FF6FB731A408282B7
:1027F000828A0A438282704721B1828A42F00202B1
:10280000828204E0828A4FF6FD731A40828270470A
:1028100002460020B1F5007F00D100BF13880B40B5
:102820000BB1012000E00020704701F40072B2F506
:10283000007F00D100BFCA430280704770B50246D6
:10284000002400230025002040F66A16B14200D182
:1028500000BFC1F3421501F01F03012606FA03F37E
:10286000012D02D19689334006E0022D02D1168A4D
:10287000334001E0968A33400C12012606FA04F434
:102880001688344013B10CB1012000E0002070BD67
:1028900010B50022002340F66A14A14200D100BF07
:1028A0000A1201249440A3B2DC43048010BD00004E
:1028B000003801400044004000480040004C004007
:1028C000005000400CB50020019000906C4800685A
:1028D00040F480306A49086000BF6948006800F42D
:1028E000003000900198401C0190009818B90198A0
:1028F000B0F5A06FF1D16248006800F4003010B16B
:102900000120009001E0002000900098012843D1B0
:102910005C48006840F010005A49086008460068AA
:1029200020F0030008600846006840F002000860DC
:102930005348406852494860084640684860084625
:10294000406840F4806048600846406820F47C108D
:1029500048600846406840F4E8104860084600684F
:1029600040F08070086000BF4548006800F00070CB
:102970000028F9D04248406820F0030040494860F0
:102980000846406840F00200486000BF3C4840688C
:1029900000F00C000828F9D10CBD10B5FFF792FF2C
:1029A00010BD10B53648006840F001003449086099
:1029B0000846406834490840314948600846006884
:1029C000324908402E4908600846006820F48020FB
:1029D00008600846406820F4FE0048604FF41F007D
:1029E0008860FFF7DAFF4FF000602949086010BDEA
:1029F00010B5002100200022214B5B6803F00C0180
:102A000021B1042906D0082928D107E0214B224C06
:102A1000236027E01F4B204C236023E0184B5B68AA
:102A200003F47010164B5B6803F48032022303EB4F
:102A3000904022B9194B4343174C23600DE0104BD3
:102A40005B6803F4003323B1144B4343124C2360FF
:102A500003E0104B4343104C236003E00D4B0E4C3E
:102A6000236000BF00BF064B5B68C3F303130C4C2D
:102A7000E15C094B1B68CB40074C236010BD000094
:102A800000100240002002400000FFF8FFFFF6FEA9
:102A900008ED00E000127A001C00002000093D0053
:102AA000200000200948804709480047FEE7FEE76C
:102AB000FEE7FEE7FEE7FEE7FEE7FEE7FEE7FEE7EE
:102AC00004480549054A064B70470000A329000841
:102AD000ED00000880090020800F0020800B0020FE
:102AE000800B002010B504462CB90120F649096876
:102AF0000882002010BDF549096808688047F2483F
:102B000000680A30F6E710B5EF480068C078F04971
:102B10004978884213DCEC480068807878B9EA4844
:102B20000068808858B9E8480068C078E6490968B4
:102B30008872E649096848688047002010BD022075
:102B4000FCE710B504462CB90120DF49096808826A
:102B5000002010BDDD49096888688047DA480068B0
:102B60000C30F6E710B5D84B1B68D978D64B1B68EC
:102B70005879D84B1B689A6990470446D248006838
:102B8000807AE8B13CB9D0480068007918B9CE48DD
:102B90000068807808B1022010BD8CB9CB49096863
:102BA000C8688047C84800684079C7490968C87242
:102BB000C5480068C078C449096808730020EBE77D
:102BC0000220E9E710B504462CB90220BE49096885
:102BD0000882002010BD0020BF490880BA48006864
:102BE000007800F07F0018BBB7490968487A00F008
:102BF000200131B1B849097841F00201B64A11709B
:102C000005E0B549097801F0FD01B34A117000F003
:102C1000400131B1B049097841F00101AE4A11706B
:102C200005E0AD49097801F0FE01AB4A11703AE0C8
:102C3000A5480068007800F07F00012801D1A6486F
:102C4000C8E7A1480068007800F07F00022828D17A
:102C50009D4A1268517901F00F0001F080027AB1AB
:102C60009E4B03EB8002D2F8002C02F03002102AB7
:102C700016D1994A127842F00102974B1A700FE070
:102C8000964B03EB8002D2F8002C02F44052B2F5CE
:102C9000805F05D1904A127842F001028E4B1A7083
:102CA00001E0002096E789490968086980478A4859
:102CB00090E72DE9F04784480068007800F07F082D
:102CC000B8F1000F0AD180480068407A00F0DF00B8
:102CD0007D49096848720020BDE8F087B8F1020F0D
:102CE0007ED179480068408818B977480068007933
:102CF00008B10220F0E7DFF8D891734800684779FF
:102D000027F080052C4670480068407900F080006C
:102D100038B1724901EB8400D0F8000C00F03006A5
:102D200006E06E4901EB8400D0F8000C00F4405638
:102D300099F80000A84204D91EB163480068807A5F
:102D400008B90220C8E707F0800080B1634901EBB1
:102D50008400D0F8000C00F0300010284BD1E0B215
:102D600001F01DF8E0B2302100F09FFE43E05B4926
:102D700001EB8400D0F8000C00F44050B0F5805F07
:102D800039D1E4B9564A92F82C10E0B201F091F82A
:102D9000524A02EB8401D1F8001C4BF68F7201EA13
:102DA000020080F4805080F4005040F4004141F073
:102DB00080014A4B03EB8402C2F8001C1BE0E0B226
:102DC00000F0D5FF454A02EB8401D1F8001C4BF618
:102DD0008F7201EA020080F4805080F4005000E01D
:102DE0000FE040F4004141F080013C4B03EB8402D2
:102DF000C2F8001C00BF35490968486980470020B7
:102E00006AE700BF022067E72DE9F0412E4800681D
:102E1000467926F080073C462B480068407900F050
:102E2000800038B12D4901EB8400D0F8000C00F08F
:102E3000300506E0294901EB8400D0F8000C00F4CD
:102E4000405523480078A04208D91F4800684088B0
:102E500020B91DB11C480068807A10B90220BDE875
:102E6000F08106F08000A0B11C4A02EB8401D1F889
:102E7000001C48F6BF7201EA020080F0100040F426
:102E8000004141F08001154B03EB8402C2F8001CA5
:102E900014E0124A02EB8401D1F8001C4BF68F7249
:102EA00001EA020080F4805040F4004141F08001CA
:102EB0000A4B03EB8402C2F8001C00BF03490968F7
:102EC000886980470020CAE73800002044000020BD
:102ED000AA0000203C0000203000002000500040EC
:102EE000AC00002010B5F7480068407A40F02000A0
:102EF000F44909684872F4490968C86980470020A4
:102F000010BD10B50246EF480068438A32B9888880
:102F1000C01AEC4C24682082002010BD08681844B8
:102F2000FBE72DE9F041E748006800F1100426882E
:102F3000A068C0B1BEB1A588B54200D93546A8B2D7
:102F4000A168884707462088401B20806088284465
:102F50006080002000F07FFF8046AAB241463846DC
:102F600000F03EFD00BF208850B14FF44050D749DB
:102F700008800021084600F07AFF3020D4490880FC
:102F80002088A188884204DB0320CE4909680872A2
:102F900018E02088002804DD0520CA490968087265
:102FA00010E0208870B90620C6490968087200211F
:102FB000C848006880B2801CC74A42F81010302010
:102FC000C3490880BDE8F0812DE9F047BD4800689D
:102FD00000F110052E88BB480068077AD6B9042F87
:102FE00018D1BE48007801280FD10021B9480068E7
:102FF00080B2801CB84A42F810103020B4490880D2
:1030000000BF0020B549087003E007271020B04931
:10301000088027E0AC88A64201D8042000E0022006
:103020000746B44200D93446A0B2A9688847804612
:10303000002000F005FF8146A2B24946404600F05C
:10304000B5FCA1B2002000F012FF2888001B2880E8
:1030500068882044688030209D49088000029B4990
:10306000088000BF974909680F72BDE8F08770B506
:10307000022694480068447892480068007800F07E
:103080007F00002844D1092C03D1FFF73CFD064600
:103090005FE0052C14D18B480068C0787F280BDCDA
:1030A00088480068807838B986480068808818B9F0
:1030B00084480068807A08B1082565E0002648E069
:1030C000032C0ED17F480068C078012807D17D48C5
:1030D0000068808818B9FFF705FF064639E0022628
:1030E00037E0012C35D177480068C07801280DD130
:1030F00074480068808848B972480068407A00F0D7
:10310000200018B1FFF7D5FD064622E0022620E098
:103110006C480068007800F07F00012805D10B2C76
:1031200017D1FFF71FFD064613E0664800680078D8
:1031300000F07F0002280BD1012C03D1FFF7B9FD6D
:10314000064606E0032C04D1FFF75EFE064600E0CB
:1031500002264EB1E0B2624A1268516988470646BB
:10316000032E01D109250FE00EB108250CE006253C
:1031700000215848006880B2801C574A42F810105D
:1031800030205349088000BF4E4909680D7270BD58
:103190002DE9F84F4B48006845780027BA46062DC0
:1031A0001BD148480068007800F07F00002813D148
:1031B000444909688878012803D149490968CF69D9
:1031C0000AE0022803D1464909680F6A04E003288F
:1031D00002D1434909684F6AADE0002D67D13948F3
:1031E00000684088002862D136480068C0880228FC
:1031F0005DD1344800680079002858D13148006812
:10320000007800F07F0030B92E480068808810B93F
:10321000AFF24F678FE02B480068007800F07F0026
:10322000012811D12749096848792D4909688A6917
:103230000021904700287ED122480068807A00282B
:1032400079D0AFF27F6776E01E480068007800F022
:103250007F0002286FD11B480068407900F00F06FC
:1032600018480068407900F07009164800684079F5
:1032700000F0800038B11B4901EB8600D0F8000C4B
:1032800000F0300806E0174901EB8600D0F8000C8A
:1032900000F4405814480078B0424CD9B9F1000FFE
:1032A00049D1B8F1000F46D0AFF2E76743E0082DEF
:1032B0001CD104480068007800F07F00D8BBAFF252
:1032C000DB7738E038000020440000204800002070
:1032D0004A000020505C00400060004032000020A6
:1032E0003C00002000500040AA0000200A2D22D1FE
:1032F000C5480068007800F07F0001281BD1C24853
:103300000068807AB8B1C0480068408898B9BE4863
:103310000068007978B9BC480068C08801280AD1E3
:10332000B94909684879B94909688A69002190470B
:1033300008B9AFF2F17757B1B3480068A0F812A00E
:10334000B148006887610020B84700240FE0AE4A0A
:1033500012685078AD4A1268116988470446032CF8
:1033600005D10920A84909680872BDE8F88FA64868
:103370000068008A4FF6FF71884204D10920A249F3
:1033800009680872F1E7022C03D09F480068008AA0
:1033900020B908209C4909680872E6E79A48006845
:1033A000007800F08000E0B397480068C088009083
:1033B00095480068008A0099884204D9924900988B
:1033C0000968088223E090480068008A8E490968ED
:1033D000C98888421BDA8C480068008A8B490968D2
:1033E00091F82C10884203DA0020894908700EE019
:1033F00085480068008A8549096891F82C1090FB7F
:10340000F1F201FB120010B90120814908707F48D8
:10341000006890F82C107C4800688182FFF7D4FD8A
:1034200007E0FFE70320784909680872000379493B
:10343000088000BF99E710B5774890F82C1000205D
:1034400000F037FD70480068007A082805D1400276
:10345000704908801020714908806B480068007A24
:10346000092801D1012010BD0020FCE738B5012456
:103470006B48006880B2001D6A4931F8100080B2C4
:1034800001EB4000009060480068007A092832D0C3
:10349000009800785C49096808700098401C00900A
:1034A000009800785849096848700098401C0090BE
:1034B000009800EB44000090009931F8020B009155
:1034C00000F0A0FE504909684880009800EB4400D5
:1034D0000090009931F8020B009100F093FE4A49E8
:1034E00009688880009800EB4400009000980088EC
:1034F00045490968C8800120434909680872424863
:103500000068C08810B9FFF7B2FD01E0FFF740FE88
:10351000FFF791FF38BD30B50146434B1A780020C4
:1035200014E00306414C04EB9353D3F8003C48F6F7
:103530008F74234048F280042343C4B2234304061B
:103540003A4D05EB9454C4F8003C401C9042E8D33B
:1035500041F08003324C241F236030BD10B52A484F
:103560000068047A022C01D0042C05D1FFF72CFD51
:1035700025480068047A1CE0062C19D1224800680E
:10358000407805280ED120480068007800F07F00C0
:1035900040B91D490968C878FFF7BDFF244909688B
:1035A000086A80471949096888688047082400E04C
:1035B0000824154909680C72FFF73DFF10BD10B5CE
:1035C00011480068047A022C01D0042C01D108248F
:1035D00012E0032C01D0052C05D1FFF7A2FC0A480C
:1035E0000068047A08E0072C05D108490968C86812
:1035F0008047082400E00824034909680C72FFF79B
:103600001AFF10BD70470000380000203C00002069
:103610003200002048000020AC0000204A000020BA
:10362000505C004000600040AA00002000500040B4
:103630004400002010B508480849086002200968C5
:1036400008720748074908600748084908600549A3
:1036500009680868804710BD00020020380000207B
:10366000AC0000203C000020DC00002044000020D2
:1036700008B50020009022E1C448008800F00F0047
:10368000C34908700846007800287CD1C14800680A
:10369000C14908800846008800F03000BF49088012
:1036A000BD48008800F44050BB490880B94909680A
:1036B0004BF6BF7201EA020080F4005080F0200057
:1036C00040F4004141F08001B24A1160AF480088E7
:1036D00000F0100090BB1046006848F60F710840DB
:1036E00011460860FFF73AFFAA4909684BF6BF7216
:1036F00001EA0200A849098801F4805109B180F467
:103700008050A549098801F4005109B180F40050A6
:10371000A249098801F0100109B180F010009F4909
:10372000098801F0200109B180F0200081B241F444
:10373000004141F08001974A116008BDFFE79548BC
:10374000006880B20090BDF8000000F40060B0B3E3
:1037500090480068C0F30E0048F68F7108408D490C
:103760000860FFF783FE8B4909684BF6BF7201EAD8
:1037700002008949098801F4805109B180F4805020
:103780008549098800E056E001F4005109B180F450
:1037900000508249098801F0100109B180F0100041
:1037A0007E49098801F0200109B180F0200081B232
:1037B00041F4004141F08001764A1160BDE7FFE726
:1037C000BDF8000000F40040002878D0714800687F
:1037D000C0F30E0048F68F7108406E490860FFF78D
:1037E000EEFE6C4909684BF6BF7201EA02006A49B5
:1037F000098801F4805109B180F480506649098834
:1038000001F4005109B180F400506449098801F0C5
:10381000100109B180F010006049098801F0200111
:1038200009B180F0200081B241F4004141F08001F3
:10383000584A116081E756480078594901EB8000E9
:10384000D0F8000C80B20090BDF8000000F40040F9
:10385000C0B14F48007801EB8000D0F8000CC0F3F5
:103860000E0048F68F710840494909784C4A02EB2E
:103870008101C1F8000C46490978491E494A52F8AD
:1038800021008047BDF8000000F08000B8B140483A
:103890000078434901EB8000D0F8000C48F60F7126
:1038A00008403B4909783E4A02EB8101C1F8000C0F
:1038B00037490978491E3C4A52F82100804735486B
:1038C0004430006880B23149088000F4004000288C
:1038D0007FF4D2AE00BF30E710B500244AE047F6CF
:1038E000FF702C49443108602848008800F00F0020
:1038F0002749087008460078294901EB8000D0F874
:10390000000C84B204F40040C8B12148007801EBF7
:103910008000D0F8000CC0F30E0048F68F7108400C
:103920001B4909781E4A02EB8101C1F8000C1849B5
:103930000978491E1B4A52F8210080471AE004F01A
:103940008000B8B112480078154901EB8000D0F82A
:10395000000C48F60F7108400D490978104A02EB37
:103960008101C1F8000C0A490978491E0E4A52F833
:103970002100804707484430006880B2034908802E
:1039800000F400400028AAD110BD0000680000200B
:1039900034000020005C0040480000204A00002065
:1039A00000500040880000206C000020F0B5144654
:1039B00004F1010C4FEA6C07DFF848C00CEB41033F
:1039C0003D460AE00678401C90F800C046EA0C220A
:1039D00023F8022B9B1C401C6D1E002DF2D1F0BD64
:1039E000F0B5561C7510074E06EB41042B4605E05A
:1039F00034F8047B20F8017B401C5B1E002BF7D1C0
:103A0000F0BD000000600040FA4908607047F948C6
:103A1000006880B27047F749091D08607047F54893
:103A2000001D006880B27047F2480830006880B21C
:103A30007047F0490C3108607047EE480C30006860
:103A400080B270474FF6F8710140EA4A10321160B7
:103A50007047E8481030006880B27047E64B03EBCF
:103A60008002C2F8001C70470146E34A02EB810065
:103A7000D0F8000C80B2704710B5DF4B03EB80022A
:103A8000D2F8002C48F68F131A400A43DA4C04EBA4
:103A90008003C3F8002C10BD0146D74A02EB810019
:103AA000D0F8000C00F4C060704730B5D24C04EB85
:103AB0008003D3F8003C48F6BF7403EA040201F027
:103AC00010030BB182F0100201F020030BB182F061
:103AD000200242F4004343F08003C74D05EB80040D
:103AE000C4F8003C30BD30B5C34C04EB8003D3F8C0
:103AF000003C4BF68F7403EA040201F480530BB1CF
:103B000082F4805201F400530BB182F4005242F46B
:103B1000004343F08003B84D05EB8004C4F8003C3B
:103B200030BD30B503460C461846FFF79DFF0546ED
:103B3000012C07D125F48050AF4A02EB8301C1F874
:103B4000000C08E0022C06D125F01000AA4A02EB76
:103B50008301C1F8000C30BD0146A74A02EB810089
:103B6000D0F8000C00F0300070470146A24A02EB8A
:103B70008100D0F8000C00F44050704710B59E4B07
:103B800003EB8002D2F8002C48F6BF7302EA03016F
:103B900081F0100181F0200141F4004242F08002E6
:103BA000954C04EB8003C3F8002C10BD10B5924B6C
:103BB00003EB8002D2F8002C4BF68F7302EA03016C
:103BC00081F4805181F4005141F4004242F08002BE
:103BD000894C04EB8003C3F8002C10BD864A02EB2D
:103BE0008001D1F8001C41F4807148F68F721140B9
:103BF00048F280021143804B03EB8002C2F8001CA4
:103C000070477D4A02EB8001D1F8001C48F68F62B4
:103C1000114048F280021143774B03EB8002C2F857
:103C2000001C7047744A02EB8001D1F8001C48F672
:103C30008F62114048F2800211436F4B03EB800208
:103C4000C2F8001C70476C4A02EB8001D1F8001CDE
:103C500041F4807148F68F72114048F2800211439E
:103C6000654B03EB8002C2F8001C7047624A02EB0E
:103C70008001D1F8001C41F4807148F68F72114028
:103C800048F2800211435C4B03EB8002C2F8001C37
:103C90007047594A02EB8001D1F8001C48F68F6248
:103CA000114048F280021143534B03EB8002C2F8EB
:103CB000001C70470146504A02EB8100D0F8000C0E
:103CC00000F03000102801D1012070470020FCE7EF
:103CD0000146494A02EB8100D0F8000C00F4405044
:103CE000B0F5805F01D1012070470020FCE7424A17
:103CF00002EB8001D1F8001CC1F30E0148F68F726F
:103D000011403D4B03EB8002C2F8001C70473A4A59
:103D100002EB8001D1F8001C48F60F721140364BBF
:103D200003EB8002C2F8001C7047334A02EB8001AB
:103D3000D1F8001C48F68F7211404CF280021143FA
:103D40002D4B03EB8002C2F8001C70472A4A02EB9D
:103D50008001D1F8001C48F68F72114048F2C00271
:103D60001143254B03EB8002C2F8001C7047224A26
:103D700002EB8001D1F8001C01F4804171B102EB2B
:103D80008001D1F8001C48F68F7211404CF280027D
:103D90001143194B03EB8002C2F8001C7047164A0E
:103DA00002EB8001D1F8001C01F0400171B102EB7F
:103DB0008001D1F8001C48F68F72114048F2C00211
:103DC00011430D4B03EB8002C2F8001C704710B585
:103DD000094B03EB8002D2F8002C48F68F731A408F
:103DE00048F280031A430A43034C04EB8003C3F8F0
:103DF000002C10BD405C0040005000400146FC4AD1
:103E000002EB8100D0F8000C00F00F00704710B5F5
:103E10004A105200F74B1B689BB203EBC003F64CF1
:103E200044F8132010BD10B54A105300F14A12682F
:103E300092B202EBC002121DEF4C44F8123010BDDA
:103E40000146EC48006880B200EBC100EA4A32F853
:103E5000100080B270470146E648006880B200EB6F
:103E6000C100001DE44A32F8100080B27047E14AF8
:103E7000126892B202EBC002921CDF4B43F81210A0
:103E8000704702463E290BDD481101F01F030BB9B4
:103E9000431E98B24FF4004343EA8023136007E0C7
:103EA000481001F001030BB1431C98B28302136068
:103EB000704710B50246CF48006880B200EBC200E0
:103EC000801DCD4C04EB40033E290BDD481101F071
:103ED0001F040CB9441EA0B24FF4004444EA8024ED
:103EE0001C6007E0481001F001040CB1441CA0B2B2
:103EF00084021C6010BD0146BE48006880B200EB21
:103F0000C100801CBC4A32F81000C0F309007047A1
:103F10000146B848006880B200EBC100801DB64A77
:103F200032F81000C0F30900704730B54B105B0049
:103F3000B04C2468A4B204EBC004AF4D45F8143073
:103F400053105C00AB4B1B689BB203EBC0031B1D03
:103F500045F8134030BD10B54A105200A54B1B6800
:103F60009BB203EBC003A44C44F8132010BD10B562
:103F70004A1053009F4A126892B202EBC002121D0F
:103F80009D4C44F8123010BD01469A48006880B23A
:103F900000EBC100984A32F8100080B27047014629
:103FA0009448006880B200EBC100001D924A32F8CC
:103FB000100080B2704730B50B46012B1FD18D49E0
:103FC000096889B201EBC001891C8B4D05EB4104E6
:103FD0003E2A0BDD511102F01F050DB94D1EA9B28D
:103FE0004FF4004545EA8125256007E0511002F0B5
:103FF00001050DB14D1CA9B28D0225600AE0022B0E
:1040000008D17C49096889B201EBC001891C7A4C4E
:1040100044F81120012B1FD17649096889B201EBC0
:10402000C001891D744D05EB41043E2A0BDD511181
:1040300002F01F050DB94D1EA9B24FF4004545EA27
:104040008125256007E0511002F001050DB14D1CDE
:10405000A9B28D0225600AE0022B08D165490968E2
:1040600089B201EBC001891D634C44F8112030BDB9
:1040700030B5034601291FD15E48006880B200EBCD
:10408000C300801C5C4D05EB40043E2A0BDD501143
:1040900002F01F050DB9451EA8B24FF4004545EAD0
:1040A0008025256007E0501002F001050DB1451C88
:1040B000A8B2850225600AE0022908D14D480068AF
:1040C00080B200EBC300801C4B4C44F8102030BD84
:1040D00030B5034601291FD14648006880B200EB85
:1040E000C300801D444D05EB40043E2A0BDD5011FA
:1040F00002F01F050DB9451EA8B24FF4004545EA70
:104100008025256007E0501002F001050DB1451C27
:10411000A8B2850225600AE0022908D13548006866
:1041200080B200EBC300801D334C44F8102030BD3A
:1041300001463048006880B200EBC100801C2E4A66
:1041400032F81000C0F309007047014629480068A2
:1041500080B200EBC100801D274A32F81000C0F386
:104160000900704701462348006880B200EBC10097
:10417000801D214A32F8100000F47C4008B1012073
:1041800070471C48006880B200EBC100801C1A4ACE
:1041900032F81000C0F3090008B10220F0E7002057
:1041A000EEE710B5012910D1114B03EB8002D2F8D4
:1041B000002C48F68F731A4048F2C0031A430C4C87
:1041C00004EB8003C3F8002C11E002290FD1084B47
:1041D00003EB8002D2F8002C48F68F731A404CF2A1
:1041E00080031A43024C04EB8003C3F8002C10BD7B
:1041F00000500040505C004000600040024641EA30
:10420000022070470146CAB20B1243EA02207047EF
:1042100000201D4908604FF43F401C4908800846B3
:1042200000881949091F0860002070472DE9F041F6
:1042300004460E46154604F07F00FFF701FE0746D0
:10424000AAB239463046FFF7B1FBA9B204F07F00AD
:10425000FFF70DFE0020BDE8F0812DE9F041044696
:104260000E46002504F07F00FFF752FE054604F0DD
:104270007F00FFF7F0FD07462A4639463046FFF734
:10428000AFFB2846BDE8F081445C004042000020BE
:104290007047012001490870704700006600002047
:1042A00010B537480068374908800846008800F490
:1042B000004035490988084008B1FFF7D9F931486D
:1042C000008800F4806030490988084030B14FF61A
:1042D000FF302B4908602D494868804729480088ED
:1042E00000F4005028490988084018B14DF6FF70C5
:1042F000234908602348008800F480502249098837
:10430000084030B14EF6FF701D490860002000F0F3
:10431000D6F91C48008800F400601B490988084051
:1043200060B11B48007810B100F0A9F902E002204A
:1043300000F0C5F94FF2FF7011490860114800887C
:1043400000F4007010490988084040B14FF6FF5052
:104350000B4908600F480078401C0E490870094856
:10436000008800F4807008490988084030B14FF691
:10437000FF6003490860072000F0A1F910BD0000AC
:10438000445C00406800002042000020AC00002097
:10439000440100206A00002010B500219548FCF778
:1043A0004DF8002094490968887200F03FF9FFF742
:1043B0002FFF00209149086010BD10B500208E49E4
:1043C000096888728C490968C8728D48C0798A4921
:1043D000096848720020FFF735FB4FF40071002098
:1043E000FFF74AFB20210020FFF75FFB1821002088
:1043F000FFF719FD58210020FFF709FD0020FFF706
:1044000011FC804890F82C100020FFF752FD7D48E9
:1044100090F82C100020FFF72AFD0020FFF7C6FBC4
:104420004FF4C0610120FFF727FB4FF4807101209A
:10443000FFF7EDFC4FF4A0710120FFF7F4FC3E21E3
:104440000120FFF714FD3E210120FFF732FD4FF45C
:1044500040510120FFF747FB30210120FFF725FBEA
:104460000020FFF758F801206449086010BD624839
:104470000068807A10B10520604908607047042008
:104480005E490860704710B55F480078092804D17C
:1044900000205D49087000F02AFB10BD70470146FE
:1044A00029B90120544A12681082002070475748E9
:1044B000FCE710B5044656492046FEF722FD10BD24
:1044C00010B5044653492046FEF71BFD10BD70B5DC
:1044D00004460025062C1AD147480068007800F0F1
:1044E0007F00012813D144480068407978B94248D8
:1044F00000688078222802D1AFF23B052BE03E48CD
:1045000000688078212826D1AFF2590523E03A4887
:104510000068007800F07F0021281CD1012C07D012
:10452000032C02D0092C14D109E0AFF28D0511E063
:10453000314800688078032800D1374D0AE02E48C2
:1045400000688078032803D109202F490870334D73
:1045500000E000BF00BF0DB9022070BD2648006812
:10456000856100212448006841820020A84700207E
:10457000F3E721480068C1782448016000207047B3
:1045800000B502461C480068007800F07F00212832
:1045900004D10B2A02D1FFF7ECFF00BD0220FCE79B
:1045A00010B504461E492046FEF7ABFC10BD10B501
:1045B00004461C492046FEF7A4FC10BD70B5054614
:1045C0000D480068C478042C01DB002070BD16483B
:1045D00000EBC4012846FEF794FCF7E702460029E9
:1045E00001DD02207047002A01DD0220FAE70020E9
:1045F000F8E700004C0000203800002040010020B7
:10460000E4A00008AC000020A8000020A4000020C6
:104610001801002010010020914800080F4A0008EE
:1046200000010020080100202001002010B5012019
:10463000FBF7B8FE01244C48046000204B49088079
:1046400008460088484908600020091D08604FF4AA
:10465000E050464908800846008843490860002029
:1046600010BD10B50120404908600020091D0860F8
:10467000FBF798FE03203C490860002010BD10B5F0
:104680003948006884B244F0080437480460006880
:1046900084B244F0040434480460FBF705FE10BD06
:1046A00010B53148006884B224F004042E48046038
:1046B000FBF701FE4FF43F402B49086010BD70B579
:1046C0000546072D01D02A4805702948007808289A
:1046D00041D2DFE800F0040A1016212E4142FFF714
:1046E000DFFF0620224908703BE0FFF7D9FF0420D6
:1046F0001F49087035E002201D49487003200870EA
:104700002FE01B484078401E194948700846407801
:1047100008B90420087024E01348006884B244F00B
:104720001004114804600520114908700A204870DF
:1047300017E00F484078401E0D4948700846407801
:1047400040B90948006884B224F0100406480460A7
:104750000620087005E000BF00BF0620044908706D
:1047600000BF00BF70BD0000405C00404200002060
:104770004501002008B501210820FCF7A7FD802095
:10478000ADF8000010208DF8030003208DF8020022
:1047900069460848FCF7DEFA08BD10B580210548D7
:1047A000FCF787FB10BD10B580210248FCF77FFBAA
:1047B00010BD0000000C01400220FB490870FB48BE
:1047C0000088A1F80100F9488078F849C97840EAE2
:1047D0004100F649097940EA8100F449497940EA03
:1047E000C100F249897940EA0110F049C97940EAEB
:1047F0004110EE49097A40EA8110EB49C870EB4854
:10480000407A08714FF47A70E8494881E649A1F886
:10481000050070470420E4490870E5480088A1F8C5
:1048200001000220C8704FF4FA60888040F21450F2
:10483000C88070470520DC490870DE480088A1F870
:104840000100DC488078C870DA48C0780871D9481F
:1048500000794871704710B5D74C2368241D216832
:10486000241D226803701C0A44701C0C84701C0EEA
:10487000C47001710C0A44710C0C84710C0EC4716B
:104880000272140A4472140C8472140EC47210BDA5
:1048900010B50446C9480068C078801E0A2871D245
:1048A000DFE800F00510111C273A4D61728524B92C
:1048B0000720C2490968088203E0FFF77DFFBA4874
:1048C00010BDA1E000BF24B90820BC4909680882D6
:1048D00003E0FFF79FFFB448F2E795E024B9062014
:1048E000B6490968088203E0FFF7A4FFAE48E7E78E
:1048F0008AE024B90420B149096808820BE0062047
:10490000A9490870AE480088A1F80100AC48807839
:10491000C8700846D4E777E024B90520A74909689C
:1049200008820BE00720A0490870A6480088A1F87B
:104930000100A4488078C8700846C1E764E024B943
:1049400005209E49096808820CE0082096490870F5
:104950009D480088A1F801009B484088A1F8030009
:104960000846ADE750E024B9382094490968088228
:1049700009E009208C49087094480088A1F80100DA
:1049800008469DE73FE03FE024B90F208B490968C6
:1049900008820BE00A20844908708D480088A1F83D
:1049A0000100C81CFFF757FF7F4889E72CE024B9B6
:1049B000342082490968088224E00B207A49087073
:1049C00084480088A1F8010082488078C870814836
:1049D0008078112804D0122807D013280FD109E0BD
:1049E0007148001D01F011FA09E06F48001D01F047
:1049F0001DF904E06C48001D01F0C2F800BF00BFC3
:104A000069485DE700E000BF00BF002058E70146AD
:104A10006A480068C078801E0A2864D2DFE800F087
:104A2000050E1B242D363F48515A21B90720634AF1
:104A30001268108201E06848704755E021B94520AE
:104A40005E4A1268108205E05C480068408A624A4B
:104A50001044F1E748E021B90820584A1268108252
:104A600001E05D48E8E73FE021B90620534A1268BB
:104A7000108201E05848DFE736E021B904204F4AB0
:104A80001268108201E05448D6E72DE021B90520D4
:104A90004A4A1268108201E04F48CDE724E021B96C
:104AA0000520464A1268108201E04B48C4E71BE02B
:104AB00021B93820414A1268108201E04648BBE71C
:104AC00012E021B90F203D4A1268108201E04248ED
:104AD000B2E709E021B93420384A1268108201E0B7
:104AE0003D48A9E700E000BF00BF0020A4E71CB5D7
:104AF00041F2111001904FF6FF7000903648B0F867
:104B00000100364908800120354908703248007894
:104B1000801E0A286CD2DFE800F005376C7D8FA07C
:104B2000A9E1E7F22C48B0F80100204908802A48A2
:104B3000C07800F0010088702748C078C0F34000BA
:104B4000C8702548C078C0F3800008712248C0783A
:104B5000C0F3C00048712048C078C0F300108871CD
:104B60001D48C078C0F34010C8711B48C078C0F31E
:104B7000801008721848007948724FF47A704881A2
:104B8000012018490870DEE01348B0F8010016490A
:104B9000088042221049C91C1348801C02F0C0FD45
:104BA000012012490870CEE06C0200201C02002097
:104BB0004A01002054010020E8F7FF1F38000020C0
:104BC0005C01002062010020660100206C010020D1
:104BD0006E01002072010020B10200207601002049
:104BE000790100204801002028020020490100200E
:104BF000A8E09E48B0F801009D4908800420887014
:104C00004FF4FA70888040F21450C880012099490E
:104C1000087098E09548B0F80100974908809348DB
:104C2000C078887091480079C870904840790871C0
:104C300001209249087086E08C48B0F80100904944
:104C400008808A48C078012800D100E000208C4903
:104C5000887001208B49087075E08448B0F8010025
:104C6000894908808148C07888706CE07F48007965
:104C7000864908700846007826280BD100220121B9
:104C80008348FDF758F901F03DF8012211468048AC
:104C9000FDF751F97D48007825281ED1012201A990
:104CA0007C4800F0A8FA012269467A4800F092FA9E
:104CB000BDF8000041F2111188420ED100BF7648C4
:104CC000006800F4E06075490843001D72490860FF
:104CD000BFF34F8F00BF00BFFEE734E06348B0F87A
:104CE00001006F4908802EE06048B0F801006D496E
:104CF00008805E48C01CFBF79CFB24E0FFE75B4894
:104D0000B0F80100684908805848C07888700846A3
:104D10008078012806D0022809D0032808D004286A
:104D20000ED10CE05148001D01F094F808E007E0B6
:104D30004E48001D01F0C1F800F073FF00E000BF15
:104D400000BF00E000BF00BF1CBD0146574A1078FD
:104D500011B90022554B1A707047554800887047AA
:104D6000544902680A6042684A6082688A607047F3
:104D7000514902680A60704710B504464F480078F0
:104D800088B10C224B49204602F09EFC58B100200D
:104D90004A4908704748016821604168616080683D
:104DA000A060012010BD0020FCE710B50446444877
:104DB000007878B144224349204602F085FC48B18E
:104DC00000203F49087044223E49204602F0A8FCDA
:104DD000012010BD0020FCE710B5044625480078EE
:104DE00078B108222249204602F06EFC48B100202A
:104DF000204908701E4801682160406860600120F9
:104E000010BD0020FCE701461C48007848B1002096
:104E10001A4A1070184802680A6080888880012049
:104E200070470020FCE710B504461648007868B1CA
:104E300004221349204602F047FC38B100201149F2
:104E400008700F4800682060012010BD0020FCE7BA
:104E500001461D48007838B100201B4A10701648E2
:104E600000680860012070470020FCE7B1020020C4
:104E70004A01002052010020540100205A01002064
:104E80005C01002060010020620100207801002008
:104E90000004004048FF00080CED00E00000FA05A7
:104EA0006C0100206E0100207201002079010020B9
:104EB000760100201C02002066010020480100202D
:104EC00049010020280200206A01002008B50121C4
:104ED0000420FCF7FBF90420ADF8000010208DF849
:104EE000030003208DF8020069461648FBF732FFE5
:104EF00004211448FBF7DBFF08BD08B5FFF7E6FF08
:104F0000FFF738FC10A002F037FB01210420FCF76A
:104F1000DDF91020ADF800008DF8030003208DF8B6
:104F2000020069460748FBF715FF10210548FBF70B
:104F3000BEFF08BD00200A490860704701200849EB
:104F400008607047000801404D454D5320435320F1
:104F5000496E6974204750494F2E200D0A00000009
:104F60009001214200B587B001210820FCF7AEF97D
:104F700001218803FCF7B7F901210846FCF7A6F9DF
:104F80004FF46040ADF8040018208DF807000320AE
:104F90008DF8060001A92C48FBF7DCFE4FF46041B8
:104FA0002948FBF784FF0020ADF808004FF4827019
:104FB000ADF80A000020ADF80C000220ADF80E009C
:104FC0000120ADF810004002ADF812001020ADF83D
:104FD00014000020ADF816000720ADF8180002A953
:104FE0001A48FCF7FDF901211848FCF79EFA18A0B1
:104FF00002F0C2FA07B000BD70B50546002405E016
:10500000601CC4B2C82C01DD002070BD02210F4815
:10501000FCF70FFB0028F3D029460C48FCF7B6FA42
:10502000002405E0601CC4B2C82C01DD0020ECE7C0
:1050300001210648FCF7FDFA0028F3D00348FCF7ED
:10504000A7FAC0B2E1E70000000C014000380040C0
:105050004D454D535F5350495F496E6974200D0AA9
:105060000000000000BF704700BF464A128802F0EF
:105070004002002AF9D0C2B2424B1B1D1A80704771
:1050800010B586B00446012144F20400FCF71EF975
:105090003C48FDF713FA4FF40070ADF814000320FC
:1050A0008DF8160018208DF8170005A93648FBF773
:1050B00051FE4FF48060ADF8140004208DF8170005
:1050C00005A93148FBF746FE01940020ADF8080021
:1050D000ADF80A00ADF80C00ADF810000C20ADF8EA
:1050E0000E0001A92748FDF72CFA012240F22551B4
:1050F0002448FDF7BEFA01212248FDF7AEFA06B0BA
:1051000010BD10B540F225511E48FDF797FB00B9C0
:1051100010BD1C48FDF712FBC4B21C48008800F407
:10512000004000B1F4E71948008800F4804060B105
:105130000A2C03D000201549088020E0134800887D
:1051400040F400401149088019E00D2C06D10F48A9
:10515000008840F480400D49088010E00B4800882A
:10516000C0F30D000A490C5408480088401C074948
:10517000088008460088C72801DD0020088000BF9D
:10518000C6E700000038014000080140800100200F
:10519000F602002010B501210C20FCF797F84FF41F
:1051A000A060FBF79DF910BD0146088870472DE906
:1051B000F04105460E461746002407E036F8141065
:1051C0002846FBF7F0FBAD1C601C84B2BC42F5DB4B
:1051D000BDE8F08130B503460C461546002207E0D5
:1051E0001846FFF7E1FF24F812009B1C501C82B206
:1051F000AA42F5DB30BD2DE9F05F80468A461746AE
:10520000B8F1006F02D33348804501D3BDE8F09F69
:10521000FBF781FAA8F1006B4FEA9B25CBF3480915
:10522000C9F50074A74200DC3C464DE04FF0006138
:1052300001EB85208A142849FFF7CCFF00260BE0FC
:1052400009EB0600244931F810004FF6FF7188423F
:1052500000D003E0701C86B2A642F1DB00BFA6427C
:105260001BDA4FF0006101EB8520FBF799FA00266D
:1052700008E03AF8160006EB0901174A22F8110077
:10528000701C86B2A642F4DB4FF0006101EB852072
:105290008A141149FFF78BFF04E02246514640462D
:1052A000FFF785FFA74200D10FE06D1C4FF000090A
:1052B0000AEB440AA044381B87B2B7F5007F02DD31
:1052C0004FF4007400E03C46B0E700BFFBF72FFA54
:1052D00000BF9BE700000108BE03002010B56FF07F
:1052E0000400FBF74CF9304800683049B0FBF1F09E
:1052F0002F4908700846007800EB4001C1EBC01050
:105300004FF6FF7101EAC0002A49088010BD002055
:105310004FF0E021086170470146264A12884A434F
:105320004FF0E0235A6100229A611A46126942F056
:1053300001021A6100BF4FF0E022106900F0010283
:105340001AB100F48032002AF5D04FF0E022126941
:1053500022F001024FF0E0231A6100229A617047A7
:105360000146134A12784A434FF0E0235A61002263
:105370009A611A46126942F001021A6100BF4FF0A9
:10538000E022106900F001021AB100F48032002A14
:10539000F5D04FF0E022126922F001024FF0E02335
:1053A0001A6100229A6170471C00002000127A00E6
:1053B000820100208401002010B5C1F3473404703D
:1053C000C1F347144470C2F3824444EAC1048470B8
:1053D000C2F38724C470C2F387040471C3F3C534D5
:1053E00044EA82144471C3F3C71484715C06240E2A
:1053F000C47110BD30B504786403457844EA45149F
:10540000857844EAD5048A4D2C6044F314040C607A
:1054100084786407E40AC57844EA8524057944EA77
:105420008504457944EA9514814D2C6044F31404B5
:1054300014604479A406E40A857944EAC514C57960
:1054400044EA65047A4D2C6044F314041C6030BDBA
:105450002DE9FE4F07460C4615461E46DDE90EAB0C
:10546000DDE90C8901207349087048707248008892
:10547000488000208880119804F028FC00B26D4913
:10548000C880284604F022FC0290204604F01EFC4E
:105490000190384604F01AFC009001466548083037
:1054A000DDE90123FFF788FF484604F00FFC029076
:1054B000404604F00BFC0190304604F007FC0090DD
:1054C00001465C481030DDE90123FFF775FF5046C7
:1054D00004F0FCFB00B257490887584604F0F6FB7D
:1054E00000B254494887109804F0F0FB00B25149CB
:1054F0008887BDE8FE8F2DE9F04F91B007A800F036
:10550000F1FF82460FAA0EA90DA800F04EF9BAF1DC
:10551000000F2DDD099804F089FA04460D4608981D
:1055200004F084FA06460F46079804F07FFA804696
:1055300042460B4641A0CDE90067CDE9024502F0A5
:105540001BF80C9804F072FA04460D460B9804F010
:105550006DFA06460F460A9804F068FA80464246FD
:105560000B463AA0CDE90067CDE9024502F004F808
:10557000314908880988491C2F4B198004F0DAFB4F
:1055800004463649099804F0E9FB05463349089872
:1055900004F0E4FB06463149079804F0DFFB0746B8
:1055A0002E490C9804F0DAFB80462C490B9804F045
:1055B000D5FB814629490A9804F0D0FB8346002296
:1055C000DDE90E0103AB17C30D983B464246494641
:1055D000CDE9006502905846FFF73AFF11B0BDE8EB
:1055E000F08F10B501211E48FCF753FFF8B10121DF
:1055F0001B48FCF75FFF10480088401C0E490880DC
:105600003E224FF480710B48FEF7D0F91549096826
:1056100048F6BF7201EA020080F0100080F020001E
:1056200040F4004141F080010E4A116000BF10BDFE
:1056300088010020BE0700208E0100206779726F6C
:105640003A25662C25662C25660A00006163633ABC
:1056500025662C25662C25660A00000000401C46A5
:1056600000040040045C004008B501210820FBF75D
:105670002DFE4FF48050ADF8000010208DF803008F
:1056800003208DF8020069466F48FBF763FB4FF477
:1056900080516D48FBF70BFC08BD70B505460C4604
:1056A00000206A4908602846FFF7A6FC2046FFF75D
:1056B000A3FC01206649C1F8B001002070BD10B5FF
:1056C000FFF7D2FF0C212120FFF7E7FF0A20FFF7A9
:1056D00023FE7C212020FFF7E0FF0A20FFF71CFEBD
:1056E0000C212320FFF7D9FF0A20FFF715FE4021E8
:1056F0002420FFF7D2FF0A20FFF70EFE0021222010
:10570000FFF7CBFF0A20FFF707FE10BD70B5044678
:10571000002500204D49086044F08000FFF76CFC34
:10572000FF20FFF769FC054601204949C1F8B00197
:10573000284670BDF8B504460D4616462820FFF7EA
:10574000E5FF8DF800002920FFF7E0FF8DF801004C
:105750009DF800009DF8011040EA012000B2208071
:105760002A20FFF7D3FF8DF800002B20FFF7CEFF94
:105770008DF801009DF800009DF8011040EA01201D
:1057800000B228802C20FFF7C1FF8DF800002D20EB
:10579000FFF7BCFF8DF801009DF800009DF8011097
:1057A00040EA012000B23080F8BD2DE9FC410446FA
:1057B0000D46164601AA911E6846FFF7BBFFBDF9CC
:1057C000020004F09FFA0746224904F0BDF9206068
:1057D000BDF90010484204F095FA07461D4904F04F
:1057E000B3F92860BDF9040004F08CFA07461949A2
:1057F00004F0AAF93060BDE8FC810FB470B504462E
:105800000D4616460E99206804F074FB20600F992F
:10581000286804F06FFB28601099306804F06AFB78
:1058200030601199206804F099FA20601599286871
:1058300004F094FA28601999306804F08FFA306007
:1058400070BC5DF814FB0000000C0140B0812142E7
:10585000008021420000204108B5FFF783FB0121B1
:105860000420FBF733FD1020ADF800008DF8030095
:1058700003208DF802006946BA48FBF76BFA102145
:10588000B848FBF714FB4FF48070ADF8000010200F
:105890008DF8030003208DF802006946B148FBF73C
:1058A00059FA08BD70B505460C460020AE4908609F
:1058B0002846FFF7A1FB2046FFF79EFB0120AB49DE
:1058C000C1F89001002070BD70B50446002500208D
:1058D000A549086044F08000FFF78EFBFF20FFF72A
:1058E0008BFB05460120A149C1F89001284670BDF7
:1058F00010B5FF24FFF7B0FF6420FFF70DFD8021F6
:105900006B20FFF7CFFF0A20FFF706FD7520FFF79A
:10591000DBFF04466420FFF7FFFC07216820FFF748
:10592000C1FF6420FFF7F8FC10216A20FFF7BAFFDF
:105930000A20FFF7F1FC02216B20FFF7B3FF0A20DA
:10594000FFF7EAFC00211A20FFF7ACFF0A20FFF75F
:10595000E3FC08211D20FFF7A5FF0A20FFF7DCFC70
:1059600018211B20FFF79EFF0A20FFF7D5FC082116
:105970001C20FFF797FF0A20FFF7CEFC10213720ED
:10598000FFF790FF204610BD2DE9FC4704460D4669
:1059900016461F46DDE90B9ADDF828803C20FFF70C
:1059A00093FF8DF800003B20FFF78EFF8DF801007C
:1059B0009DF800009DF8011040EA012000B220800F
:1059C0003E20FFF781FF8DF802003D20FFF77CFFAE
:1059D0008DF803009DF802009DF8031040EA0120B5
:1059E00000B228804020FFF76FFF8DF804003F20B1
:1059F000FFF76AFF8DF805009DF804009DF805107B
:105A000040EA012000B230804220FFF75DFF8DF8B0
:105A100000004120FFF758FF8DF801009DF80000BD
:105A20009DF8011040EA012000B2AAF800004420CD
:105A3000FFF74AFF8DF800004320FFF745FF8DF880
:105A400001009DF800009DF8011040EA012000B21D
:105A500038804620FFF738FF8DF802004520FFF719
:105A600033FF8DF803009DF802009DF8031040EA13
:105A7000012000B2A8F800004820FFF725FF8DF8AC
:105A800004004720FFF720FF8DF805009DF8040073
:105A90009DF8051040EA012000B2A9F80000BDE819
:105AA000FC872DE9F04788B00546002407A805A922
:105AB0008A1E04ABCDE900210290821E06A9801F38
:105AC000FFF762FF00BF14E00DF1160131F9140079
:105AD00004F018F907464FF0814104F03FF90646FB
:105AE0004FF08E4104F030F805F10C0141F824002C
:105AF000641C032CE8DB00241FE004A931F9140026
:105B000004F000F982461A4850F82410504604F078
:105B1000F1F98146174904F021F98046164904F04D
:105B20001DF907464FF08E4104F00EF80646134962
:105B300004F00AF845F82400641C032CDDDBBDF9F1
:105B40001C0042F21071484348F26B2190FBF1F0C7
:105B500000F63406304604F0D5F8686208B0BDE8B7
:105B6000F08700000008014090012142000021421E
:105B700004080020DB0F49400000FA4400003443D1
:105B80002DE9F0410546002400271822E649E748A0
:105B9000FFF720FB00BF06E0E34830F81400FF28C1
:105BA00000D17F1C641C182CF6DB182F18D10024A0
:105BB00013E00021DE4840F824104FF07E5104EB42
:105BC00044020C3000EB820040F82410002045F81D
:105BD0002400E01C45F82010641C032CE9DB1EE0C7
:105BE000D14E002404E056F8240045F82400641C3B
:105BF000062CF8DB002410E056F82410CC4840F8BE
:105C00002410E01C56F8201004EB4402C8480C3065
:105C100000EB820040F82410641C032CECDBBDE890
:105C2000F08110B5C348FFF7ABFF10BD70B5044657
:105C30000622BD49BD480838FFF7CCFABA4D28689E
:105C4000206068686060A868A06070BD10B5BA4840
:105C5000FFF7ECFF10BD70B505460024B24EB61C30
:105C600041F21110B11E088000BF05E0281D50F858
:105C7000240046F82400641C032CF7DB0722AA4901
:105C8000AA481038FFF7B7FA70BD3EB505460024A4
:105C900000200090019002900722A349A3481038E9
:105CA000FFF798FAA04800884FF6FF7188420CD1A0
:105CB00000BF04E00021281D40F82410641C032CC0
:105CC000F8DB2846FFF7C7FF11E09748801C0090DB
:105CD000001D0190001D0290002406E05DF82400E4
:105CE0000168281D40F82410641C032CF6DB3EBD1F
:105CF00010B58F481C38FFF7C8FFFFF7A7FFFFF765
:105D000090FF10BD2DE9F04F89B0002004460546F4
:105D100000210E460F46884689468346824635E076
:105D200004AA06A8811E05ABCDE90102009108AACC
:105D3000811D07A8FFF728FEBDF9140003F08BFBB7
:105D400022462B46CDE9020103F042F904460D46F6
:105D5000BDF9160003F07FFB32463B46CDE9020158
:105D600003F036F906460F46BDF9180003F073FB41
:105D700042464B46CDE9020103F02AF980468946A6
:105D80000BF1010B0AF101001FFA80FABAF5FA6F64
:105D9000C6DB584603F05FFB02460B46CDE9000127
:105DA0002046294603F0D0F9CDE9020103F0DEF8E0
:105DB0005F491C394860584603F04DFB02460B46CC
:105DC000CDE900013046394603F0BEF9CDE90201C4
:105DD00003F0CCF856491C398860584603F03BFB69
:105DE00002460B46CDE900014046494603F0ACF9B6
:105DF000CDE9020103F0BAF84D491C39C8600846E4
:105E0000FFF729FF09B0BDE8F08F70B504460722FF
:105E1000454946481038FFF7DDF9434DAD1C286869
:105E2000206068686060A868A06070BD10B500243C
:105E300000BF06E04FF6FF703B4921F81400601CDC
:105E4000C4B2072CF6DB0722374938481038FFF771
:105E5000D2F910BD70B50446334DAD1C20682860E2
:105E600060686860A068A8600722A91E2F481038E3
:105E7000FFF7C1F970BD0EB50020009001900290AF
:105E80006846FFF7E7FF0EBD70B50446264D206853
:105E9000286060686860A068A860062229462348D8
:105EA0000838FFF7A8F970BD0EB5002000900190EA
:105EB00002906846FFF7E8FF0EBD70B50546002664
:105EC000194C2868206068686060A868A060E8686D
:105ED000E0602869206168696061182221461348E2
:105EE000FFF789F900BF10E054F82610104840F879
:105EF0002610F01C54F8201006EB46020C480C301B
:105F000000EB820040F82610761C032EECDB70BDFF
:105F100000B587B01822094901A801F046FC01A884
:105F2000FFF7CBFF07B000BD6408002010FF00089A
:105F30001C0800209001002058080020F0A2000852
:105F40007FB505460C4601210220FBF7CCF9ADF8E0
:105F50000850ADF804400020ADF80A00ADF8060086
:105F600001A93248FBF770FC012211462F48FBF7CC
:105F7000E2FF1D208DF8000000208DF801000320B5
:105F80008DF8020001208DF803006846FAF7ADFA9B
:105F900001212648FBF7B4FF7FBD0EB50121042087
:105FA000FBF7A1F94FF6FF70ADF804004720ADF8FC
:105FB00000000020ADF80600ADF8020069461C485C
:105FC000FBF742FC01211A48FBF79AFF0121084622
:105FD000FBF789F94FF6FF70ADF804004720ADF8E4
:105FE00000000020ADF80600ADF8020069464FF051
:105FF0008040FBF729FC01218807FBF781FF0EBDDC
:1060000070B500240A48243000880A49086000203E
:106010000749243108800748006803F08BFE0546D5
:10602000054903F091FD0446204670BD0004004080
:1060300000080040A80100200024F4492DE9F041A7
:106040000746884614460F2C03DD4FF0FF30BDE8AD
:10605000F081FEF76FFF47F08000FEF7CDFF0026CE
:1060600006E00020FEF7C8FF0546FE488555761C71
:10607000A642F6DBFEF762FF2246FA49404601F0EF
:106080004FFB0020E3E7F8B505460C46FEF752FF4C
:106090002E463046FEF7B0FF07462046FEF7ACFF1F
:1060A0000746012269462846FFF7C8FFFEF746FF6C
:1060B0009DF80000A04201D10120F8BD6FF0010061
:1060C000FBE710B50446E8480078A04201D1012062
:1060D00010BDE548047021467620FFF7D4FFF7E7AE
:1060E00010B50020FFF7EDFFE0A001F045FA012117
:1060F0001120FFF7C8FF04460120FFF70DF910BD7E
:1061000038B504460020FFF7DCFF01226946502025
:10611000FFF794FF002802DA4FF0FF3038BD9DF8FA
:10612000000064F35F10C0B200909DF80010502092
:10613000FFF7A9FF002802DA6FF00100EEE7C4F1D3
:106140000402012101FA02F003F0DCFD05464FF0E4
:106150008E4103F0F9FCCA490860CA480470CAA01D
:1061600001F00AFA0120D9E7F8B504460020FFF74C
:10617000A8FF012269464F20FFF760FF002802DADE
:106180004FF0FF30F8BD9DF8000064F35F10C0B21F
:1061900000909DF800104F20FFF775FF002802DAED
:1061A0006FF00100EEE7012101FA04F003F0AAFD0F
:1061B00006463146BA4803F0C7FC05464FF08E410B
:1061C00003F0C2FCB7490860B74804700120D9E762
:1061D00070B504460D460120FFF773FF002802DA70
:1061E0004FF0FF3070BD012C07D100210B20FFF7CD
:1061F0004AFF00280ADAE01EF4E703210B20FFF72C
:1062000042FF002802DA6FF00200EBE70220FFF7FE
:1062100058FF002802DA6FF00300E3E7012D07D1F1
:1062200000210320FFF72FFF00280ADAA81FD9E773
:1062300001210320FFF727FF002802DA6FF0050095
:10624000D0E70020FFF73DFF002802DA6FF00600DC
:10625000C8E70120C6E72DE9FF4100240E2293493B
:106260001D20FFF7EBFE002803DA601E04B0BDE836
:10627000F08100240DE0012000EB44008B49085C14
:1062800011F8141040EA012000B22DF81400601C2F
:10629000C4B2072CEFDBBDF9000003F033FD064666
:1062A00083480168304603F04FFC05468148016889
:1062B000284603F0E7FB80490860BDF9020003F0BF
:1062C00021FD07466E480168384603F047FD064643
:1062D0007A480168304603F00DFE054678480168AB
:1062E000284603F03BFD77490860BDF9040003F040
:1062F00009FD074662480168384603F02FFD06464F
:106300006E484168304603F0F5FD05466C4841682B
:10631000284603F023FD6B494860BDF9060003F0F1
:10632000F1FC074656480168384603F017FD06465B
:1063300062488168304603F0DDFD054660488168AB
:10634000284603F00BFD5F498860BDF9020003F0A9
:10635000D9FC064659480168304603F0CBFD054696
:1063600057480168284603F0F9FC57490860BDF911
:10637000040003F0C7FC064650484168304603F06D
:10638000B9FD05464E484168284603F0E7FC4E49F2
:106390004860BDF9060003F0B5FC06464748816831
:1063A000304603F0A7FD054645488168284603F0BE
:1063B000D5FC45498860BDF9080003F0A3FC0646FA
:1063C00038480168304603F0C9FC05463F4801687B
:1063D000284603F08FFD3E490860BDF90A0003F02E
:1063E00091FC06462F480168304603F0B7FC05468D
:1063F00036484168284603F07DFD35494860BDF9BF
:106400000C0003F07FFC064626480168304603F086
:10641000A5FC05462D488168284603F06BFD2C49F4
:106420008860BDF9080003F06DFC05462748016847
:10643000284603F05FFD27490860BDF90A0003F014
:1064400061FC054621484168284603F053FD214977
:106450004860BDF90C0003F055FC05461B488168F7
:10646000284639E0EE010020FE01002049434D2D71
:106470003432363838502052657365742E0D0A0058
:10648000D4010020DC010020736574207365744121
:106490006363656C4653207375636573732E0A00DE
:1064A0000000FA44D8010020DD0100200C09002082
:1064B000B8010020BC010020CC010020A008002071
:1064C000C0010020C4080020DC08002000090020D2
:1064D000D0080020E808002003F00CFDFE49886089
:1064E0000120C3E62DE9FF4104460E22FB491D2091
:1064F000FFF7A4FD002804DA4FF0FF3004B0BDE838
:10650000F08100200DE0012101EB4001F34A515CD4
:1065100012F8102041EA022109B22DF81010411C96
:10652000C8B20728EFDBBDF9000003F0EBFB06461D
:10653000EB480168304603F007FB0546E94801686F
:10654000284603F09FFAE8490860BDF9020003F00D
:10655000D9FB0746E5480168384603F0FFFB0646CD
:10656000E3480168304603F0C5FC0546E148016890
:10657000284603F0F3FBE0490860BDF9040003F08E
:10658000C1FB0746D9480168384603F0E7FB0646D9
:10659000D7484168304603F0ADFC0546D548416810
:1065A000284603F0DBFBD4494860BDF9060003F040
:1065B000A9FB0746CD480168384603F0CFFB0646E5
:1065C000CB488168304603F095FC0546C948816890
:1065D000284603F0C3FBC8498860BDF9020003F0F8
:1065E00091FB0646C2480168304603F083FC05462D
:1065F000C0480168284603F0B1FBC0490860BDF9F6
:10660000040003F07FFB0646B9484168304603F0BA
:1066100071FC0546B7484168284603F09FFBB7491F
:106620004860BDF9060003F06DFB0646B04881687E
:10663000304603F05FFC0546AE488168284603F00B
:106640008DFBAE498860BDF9080003F05BFB064690
:10665000AB480168304603F081FB0546A948016854
:10666000284603F047FCA8490860BDF90A0003F07A
:1066700049FB0646A2480168304603F06FFB054619
:10668000A0484168284603F035FC9F494860BDF9A1
:106690000C0003F037FB064699480168304603F0CA
:1066A0005DFB054697488168284603F023FC964920
:1066B0008860BDF9080003F025FB05468E48016897
:1066C000284603F017FC84490860BDF90A0003F06E
:1066D00019FB054688484168284603F00BFC7E49B3
:1066E0004860BDF90C0003F00DFB05468248816847
:1066F000284603F0FFFB7849886000200DE07E49C2
:1067000051F8202004F10C0141F820207E4951F875
:10671000201044F82010411CC8B20328EFDB724857
:10672000006860620120E9E62DE9F0410024774825
:1067300005780320FFF718FD002802DA601EBDE887
:10674000F0810020724908604860886000244BE0B6
:10675000FFF781FD6F48006803F0D4FA0746694AE5
:106760001168694A106803F08DF98046394603F0D4
:10677000EBF9064666480168304603F083F9644940
:1067800008606448006803F0BDFA07465D4A516836
:106790005D4A506803F076F98046394603F0D4F933
:1067A00006465B484168304603F06CF9584948603A
:1067B0005848006803F0A6FA0746524A9168524AC0
:1067C000906803F05FF98046394603F0BDF906464C
:1067D0004F488168304603F055F94D4988600120E3
:1067E000FEF79AFD601CC4B24A4800688442AFDBE1
:1067F0004748006843490860454840684860444845
:10680000806888602846FFF7AFFC002802DA6FF046
:10681000030094E7012092E72DE9F04F8BB0074683
:106820008846934601200A9000BF00BF76200A994F
:10683000FFF729FC0022384B3846414602F072FE31
:10684000CDE9080135483649DDE9082302F06AFE42
:106850000022344BCDE9040102F076FCCDE90601BB
:1068600002F0D6FA05460E4626F0004000222E4BD6
:10687000CDE906502846079902F018FE11D80022EB
:106880002A4B2846314602F04DFECDE9040102F0C4
:106890000DFBCDE9060102F0AFFD04B24FF0000A96
:1068A00078E04FF0010A00221F4B2846314602F0E3
:1068B00037FF4DD22A46334600201D4902F0CCFF57
:1068C00000221C4BCDE9000102F02CFE0022174BE8
:1068D000CDE9020130E00000E80800200C090020AA
:1068E000B8010020BC010020CC010020D401002010
:1068F000A0080020C0010020C4080020DC080020FF
:10690000D801002000090020D0080020DD0100206F
:10691000F4080020D001002000408F401F85EB517B
:10692000B81E1940000040400000EC3F00007040DD
:106930000000F03F0000204002F0F4FDCDE904012A
:1069400002F0B4FACDE9060102F056FD04B221E0EE
:106950000022F94B2846314602F0A8FD1AD22A46F9
:1069600033460020F54902F033FB0022F44BCDE919
:10697000000102F0D7FD0022F24BCDE9020102F046
:10698000D1FDCDE9040102F091FACDE9060102F052
:1069900033FD04B2BBF1000F18D1EB4800786AF365
:1069A000C300E9490870210AE748007861F3000054
:1069B000E5490870E1B20F20FFF765FBDFF8889327
:1069C00099F800101220FFF75EFB72E0BBF1020F96
:1069D00018D1DD4800786AF30410DB490870210AF9
:1069E000D948007861F34100D7490870E1B210201E
:1069F000FFF749FBDFF8509399F800101220FFF7DA
:106A000042FB56E0BBF1040F18D1CF4800786AF37F
:106A10004510CD490870210ACB48007861F3820007
:106A2000C9490870E1B21120FFF72DFBDFF8189378
:106A300099F800101220FFF726FB3AE0BBF1050F92
:106A400037D1C14800786AF3C300BF490870210AF2
:106A5000BD48007861F30000BB4908700846007823
:106A60006AF304100870210AB748007861F3410006
:106A7000B5490870084600786AF345100870210A85
:106A8000B148007861F38200AF490870E1B20F208D
:106A9000FFF7F9FAE1B21020FFF7F5FAE1B21120A1
:106AA000FFF7F1FADFF8A09299F800101220FFF733
:106AB000EAFA00200A9076200A99FFF7E4FA0BB070
:106AC000BDE8F08F70B50446012529467620FFF712
:106AD000DAFA012000EB0410C6B231461320FFF7AA
:106AE000D2FA002529467620FFF7CDFA70BD70B5A1
:106AF00004460126012C06D19448007820F00100BC
:106B00009249087006E09148007820F00100401C8E
:106B10008E49087031467620FFF7B5FA8A4D2978FC
:106B20000B20FFF7B0FA002631467620FFF7ABFACC
:106B300070BD2DE9F04107460C464FF0000804FBFC
:106B400004F6002F77D14FF0010841467620FFF779
:106B50009AFA21460C20FFF796FAF1B20D20FFF7C2
:106B600092FA310A7A48007861F303007849087094
:106B7000012C06D10846007820F0F000F0300870B3
:106B80007DE0022C07D17248007820F0F000D03070
:106B90006F49087073E0032C07D16D48007820F02E
:106BA000F000C0306A49087069E0042C07D16848D9
:106BB000007820F0F000B030654908705FE0052CE7
:106BC00001D0062C07D16248007820F0F000A030F8
:106BD0005F49087053E0062C09DD0A2C07DA5C488F
:106BE000007820F0F00090305949087047E0092CF7
:106BF00009DD0E2C07DA5648007820F0F0008030CE
:106C0000534908703BE00D2C09DD132C07DA50487E
:106C1000007820F0F00070304D4908702FE0122C01
:106C20000ADD1B2C08DA4A48007820F0F0006030BA
:106C30004749087023E02EE01A2C09DD252C07DADD
:106C40004348007820F0F00050304149087016E0C9
:106C5000242C09DD352C07DA3D48007820F0F000BF
:106C600040303B4908700AE0352C08DD3F2C06DC3B
:106C70003748007820F0F000303035490870344D46
:106C800029780E20FFF7FFF94FF0000841467620E3
:106C9000FFF7F9F911E2012F78D14FF002084146D0
:106CA0007620FFF7F0F92B48007864F34600294975
:106CB00008700D4629780320FFF7E5F9F1B20420AA
:106CC000FFF7E1F9310A2448007861F30300224913
:106CD0000870012C06D10846007820F0F000F03052
:106CE00008708FE0022C07D11B48007820F0F000DC
:106CF000D0301949087085E0032C07D11648007878
:106D000020F0F000C030144908707BE0042C07D15B
:106D10001148007820F0F000B0300F49087071E0A1
:106D2000052C01D0062C19D10B48007820F0F0007A
:106D3000A0300949087065E00000ECBF0000F03F9A
:106D4000000020C000007040AC010020AE01002017
:106D5000AD010020AF010020B0010020062C09DDAC
:106D60000A2C07DAFD48007820F0F0009030FB494B
:106D7000087047E0092C0ADD0E2C08DAF748007885
:106D800020F0F0008030F54908703BE046E00D2C23
:106D900009DD132C07DAF148007820F0F00070309C
:106DA000EE4908702EE0122C09DD1B2C07DAEB48A7
:106DB000007820F0F0006030E849087022E01A2CDA
:106DC00009DD252C07DAE548007820F0F000503086
:106DD000E249087016E0242C09DD352C07DADF487B
:106DE000007820F0F0004030DC4908700AE0352CD3
:106DF00008DD3F2C06DCD948007820F0F000303068
:106E0000D6490870D54D29780520FFF73CF94FF099
:106E1000000841467620FFF736F94EE1052FFCD1F8
:106E20004FF0010841467620FFF72DF921460C204E
:106E3000FFF729F9F1B20D20FFF725F9310AC8480B
:106E4000007861F30300C6490870012C06D108469A
:106E5000007820F0F000F03008707CE0022C07D1C0
:106E6000BF48007820F0F000D030BD49087072E0D3
:106E7000032C07D1BA48007820F0F000C030B849A0
:106E8000087068E0042C07D1B548007820F0F000C5
:106E9000B030B34908705EE0052C01D0062C07D154
:106EA000AF48007820F0F000A030AD49087052E003
:106EB000062C09DD0A2C07DAA948007820F0F0003A
:106EC0009030A749087046E0092C09DD0E2C07DA3E
:106ED000A348007820F0F0008030A14908703AE023
:106EE0000D2C09DD132C07DA9D48007820F0F00006
:106EF00070309B4908702EE0122C09DD1B2C07DA3C
:106F00009748007820F0F00060309549087022E042
:106F10001A2C09DD252C07DA9148007820F0F000C2
:106F200050308F49087016E0242C09DD352C07DA23
:106F30008B48007820F0F0004030894908700AE062
:106F4000352C08DD3F2C06DC8548007820F0F00069
:106F5000303083490870824D29780E20FFF793F86E
:106F60004FF0020841467620FFF78DF87D48007803
:106F700064F346007B4908700D4629780320FFF72B
:106F800082F8F1B20420FFF77EF8310A73480078E6
:106F900061F3030071490870012C06D1084600789E
:106FA00020F0F000F03008707CE0022C07D16B4834
:106FB000007820F0F000D0306849087072E0032CAF
:106FC00007D16648007820F0F000C03063490870AF
:106FD00068E0042C07D16148007820F0F000B03060
:106FE0005E4908705EE0052C01D0062C07D15B4895
:106FF000007820F0F000A0305849087052E0062CCC
:1070000009DD0A2C07DA5548007820F0F0009030AE
:107010005249087046E0092C09DD0E2C07DA4F486A
:10702000007820F0F00080304C4908703AE00D2CD8
:1070300009DD132C07DA4948007820F0F0007030A1
:10704000464908702EE0122C09DD1B2C07DA434854
:10705000007820F0F00060304049087022E01A2CDF
:1070600009DD252C07DA3D48007820F0F00050308B
:107070003A49087016E0242C09DD352C07DA374828
:10708000007820F0F0004030344908700AE0352CD8
:1070900008DD3F2C06DC3148007820F0F00030306D
:1070A0002E4908702D4D29780520FEF7ECFF4FF092
:1070B000000841467620FEF7E6FFBDE8F0812DE9A5
:1070C000F04105460E460027D5B9012E06D12648C7
:1070D000007820F002002449087006E02248007879
:1070E00020F00200801C20490870012739467620D4
:1070F000FEF7C9FF1C4C21780B20FEF7C4FF57E0B8
:10710000012D1AD1012E06D11648007820F0010079
:107110001449087006E01348007820F00100401C74
:1071200010490870022739467620FEF7ACFF0D4C57
:1071300021780320FEF7A7FF3AE0052D38D1012E74
:1071400014D10948007820F002000749087005486A
:10715000007820F001000349087015E0B00100201C
:10716000AD010020AF010020AE010020C948007829
:1071700020F00200801CC7490870C748007820F042
:107180000100401CC4490870012739467620FEF7EB
:107190007AFFC04C21780B20FEF775FF0227394695
:1071A0007620FEF770FFBC4C21780320FEF76BFFC2
:1071B000002739467620FEF766FFBDE8F0812DE90D
:1071C000F04107460D4616464FF000080020FEF736
:1071D00078FF032D01DC0F2E02DD4FF0FF3858E061
:1071E000B7B9AE48007865F38300AC4908700C4627
:1071F00021785120FEF747FFA948007866F3030085
:10720000A74908700C4621785220FEF73CFF40E069
:10721000012F16D1A348007865F3C400A149087076
:107220000C4621785320FEF72EFF9D48007866F328
:1072300007109B4908700C4621785220FEF723FF67
:1072400027E0052F25D19548007865F38300934901
:1072500008700C4621785120FEF715FF9148007800
:1072600065F3C4008F4908700C4621785320FEF75F
:107270000AFF8B48007866F30300894908700846C6
:10728000007866F3071008700C4621785220FEF74C
:10729000FAFE4046BDE8F0812DE9F04107460D4673
:1072A00014464FF000080020FEF70BFF002F3CD1E2
:1072B0000F2D01DC072C02DD4FF0FF3867E07A4824
:1072C000007865F30300784908700846007864F395
:1072D000471008700E4631784F20FEF7D4FE082C78
:1072E00022D2DFE804F00405090D1115191D1BE079
:1072F0000020FEF739FF17E00120FEF735FF13E00D
:107300000220FEF731FF0FE00320FEF72DFF0BE018
:107310000420FEF729FF07E00520FEF725FF03E024
:107320000620FEF721FF00BF31E0012F2FD10F2DE6
:1073300001DC032C02DD6FF0010828E05B480078D7
:1073400065F30300594908700846007864F3471054
:1073500008700E4631785020FEF795FE34B1012CAE
:1073600008D0022C0AD0032C10D10BE00020FEF72D
:10737000C7FE0BE00120FEF7C3FE07E00220FEF788
:10738000BFFE03E00320FEF7BBFE00BF00BF404688
:10739000BDE8F08110B50024FEF7A2FE0020FEF744
:1073A00090FE012242497520FEF748FE40480078D1
:1073B000472806D03E4801783EA000F0DDF8E01EE8
:1073C00010BD3B48017845A000F0D6F80F214E20B3
:1073D000FEF759FE002802DA6FF00300F0E7002004
:1073E000FEF78EFE0446002C01DA2046E8E7002076
:1073F000FEF7BAFE0446002C01DA2046E0E7012041
:10740000DEE710B5FFF7C6FF0446002C0EDA3FA0FA
:1074100000F0B2F843A000F0AFF8214649A000F018
:10742000ABF83EA000F0A8F8002010BD49A000F085
:10743000A3F8052200204E49FFF7EEF90120FFF7DF
:1074400041FB0120FFF753FB06210020FFF771FBF2
:1074500001210020FFF733FE012202210020FFF767
:10746000AEFE01220F210020FFF716FF06210120AA
:10747000FFF75FFB01210846FFF721FE07220221EB
:107480000120FFF79CFE01220F211046FFF704FFA9
:107490000120CAE7AE010020AF010020B1010020A9
:1074A000B2010020B4010020B3010020B50100208A
:1074B0000C090020526561642049434D343236384E
:1074C00038206572726F722C2052656164204944C5
:1074D000203D202578200A0D0000000052656164DF
:1074E0002049434D3432363838204944207375637F
:1074F0006573732C2049434D343236383820494463
:10750000203D2030782578200A0D0000494D55B3E4
:10751000F5CABCBBAFB2BBB3C9B9A620200D0A20C7
:1075200000000000BCECB2E9494D55BDD3CFDFBB34
:10753000F2B3A2CAD4D1ADBBB7B9A9B5E720200D2B
:107540000A200000B4EDCEF3D7B4CCAC3A256420C9
:107550002020200049434D2D343236383820696EC2
:107560006974207375636573732E200D0A00000023
:107570000000F03F704700000FB4044910B503AAA3
:10758000029800F0B9FB10BC5DF814FB7C010020F0
:107590002DE9F0410E460446002020622046E168B5
:1075A000884730B3252805D0D4E901219047206AC7
:1075B000401CF2E7E168204600278847050018D004
:1075C000A5F14100192802D820354FF40067324652
:1075D000294620462760F8F7E3FD40B1012804D092
:1075E000F61D26F007060836D8E7361DD6E72846EA
:1075F000DAE7206ABDE8F0812DE9F0410646002473
:1076000010687529314616A510D0AFF30080002808
:1076100002DA404213A507E031688A0701D512A5B6
:1076200002E0490704D511A5012401E0AFF3008071
:1076300000210A2206F1240709E0B0FBF2FCB0FBAE
:10764000F2F302FB1C00303078541846491C002825
:10765000F3D123462A463046BDE8F04100F0E6B8B3
:10766000000000002D0000002B00000020000000A2
:1076700070B504460D4621461068AFF3008021889E
:10768000090502D50F4A7A4402E00E4A7A440E32C6
:10769000002104F1240305E000F00F060009965DC7
:1076A0005E54491C0028F7D120780023000704D538
:1076B000702D02D009B1022311322046BDE870407E
:1076C00000F0B4B87E2C000040EA010310B59B071F
:1076D0000FD1042A0DD310C808C9121F9C42F8D03C
:1076E00020BA19BA884201D9012010BD4FF0FF30ED
:1076F00010BD1AB1D30703D0521C07E0002010BD03
:1077000010F8013B11F8014B1B1B07D110F8013B8E
:1077100011F8014B1B1B01D1921EF1D1184610BD6F
:10772000032A40F2308010F0030C00F0158011F8AD
:10773000013BBCF1020F624498BF11F801CB00F885
:10774000013B38BF11F8013BA2F1040298BF00F8D9
:1077500001CB38BF00F8013B11F0030300F0258096
:10776000083AC0F0088051F8043B083A51F804CBBD
:10777000A0E80810F5E7121D5CBF51F8043B40F883
:10778000043BAFF30080D20724BF11F8013B11F88E
:1077900001CB48BF11F8012B24BF00F8013B00F8D2
:1077A00001CB48BF00F8012B704710B5203AC0F05C
:1077B0000B80B1E81850203AA0E81850B1E81850F2
:1077C000A0E81850BFF4F5AF5FEA027C24BFB1E82F
:1077D0001850A0E8185044BF18C918C0BDE81040A0
:1077E0005FEA827C24BF51F8043B40F8043B08BFA9
:1077F0007047D20728BF31F8023B48BF11F8012B70
:1078000028BF20F8023B48BF00F8012B70477047A3
:1078100070477047704710B500F084FA006810BDDB
:1078200010B5044600F07EFA046010BD2DE9F04763
:107830000D4699469246044600F1240801688806E0
:1078400004D5E06921F01001216000E00120A84288
:1078500001DD471B00E00027A1697A1902EB09004E
:10786000081AA0612078C00602D42046AFF3008039
:10787000002608E0D4E901211AF806009047206AA2
:10788000401C761C20624E45F4DB2078C0060AD5E9
:107890002046AFF3008006E0D4E901213020904774
:1078A000206A401C2062381EA7F10107F4DC07E0C3
:1078B000D4E9012118F805009047206A401C206295
:1078C000281EA5F10105F3DC2046AFF300802078E7
:1078D000000602D50220BDE8F0870120FBE77047D3
:1078E0002DE9FF4F0C461E464FF0FF378BB0D2E913
:1078F0000001DDF860800A908A46C1F30A5505B997
:107900003D46002108464FF00000BAF1000F00F498
:10791000400005DA00EB80004FF4400101EA50001E
:107920004FEA9059B9F1010F00DDB9460A9850EAC3
:107930004A000ED044F61050A5F2FF3545432F14EF
:10794000B8F1000F1ED07542291E1EDDC9F10002DC
:107950001CE0B8F1010F4FF0000001D0302103E02E
:10796000F24305E02154401CB042FBDB30460022CC
:10797000002121540B99C1F80880C1E900200FB003
:10798000BDE8F08FBD1B6D1CDEE74A4600DA694298
:1079900006A800F069FA06AB93E8070003AB83E89A
:1079A000070050460A9900F043FB8DE80700A0F558
:1079B00000501F3800900398002D09DD42F21F018E
:1079C0004A46084403A90390684600F0A2FD08E077
:1079D000A0F500504A461F3803A90390684600F0FE
:1079E000ACFD8DE807000004000C03D04FF0FF3021
:1079F000410800E01046B8F1000F03D000220092C9
:107A000015461EE0751E05D400F090F9303262551F
:107A10006D1EF9D5B3460122084302D000227F1C17
:107A200004E02078302801D100227F1E002A099727
:107A300086D01DE0112D07DA00F078F9303262555A
:107A40006D1C50EA0102F5D1084302D00098C8B17C
:107A50000EE00021681E05E0235C625C6354225442
:107A6000401E491C8142F7DBAB46A81B401E099013
:107A7000002004F80B000B98099AC0F80880C0E9B0
:107A8000002B7CE711264FF0000859E72DE9F04F55
:107A900088460446D21D22F0070191B0D1E90001C9
:107AA000CDE90A0100F07FFE02460B98C00F01D01D
:107AB0002D2007E02068810701D52B2002E020213E
:107AC00001EAC000032A099001D0072A05DB03461A
:107AD0004146204600F088F90BE12078800601D568
:107AE000E06900E00620B8F1650F814606D0B8F1E4
:107AF000660F18D0B8F1670F70D131E00020B9F1EE
:107B0000110F009001DB112301E009F101030AAA22
:107B100001A90CA8FFF7E4FEDDE90C70002609F1CD
:107B20000105834647E001204B4600904FF0004797
:107B30000AAA01A90CA8FFF7D3FEDDE90DB00C9944
:107B40005D46002610B909F101000D18B9EB0500DA
:107B500003D4C0F1FF3609F10105A5EB09002BE0C4
:107B6000B9F1010F01DA4FF001090020B9F1110F4D
:107B70000090484601DD112300E003460AAA01A94E
:107B80000CA8FFF7ADFEDDE90C704D4600268346DC
:107B9000207800070AD4AB4500DA5D4601A8012D24
:107BA00004DD411911F8011C302907D04F4502DAD4
:107BB00017F1040F04DA012082460FE06D1EEEE794
:107BC000002F02DCED1B3E4403E0781CA84200DDE0
:107BD0007D1CB81B00F1010A4FF000472078000718
:107BE00003D4AA4501DB4FF0FF3A0021B7F1004F63
:107BF0000DF143088DF8431024D002202B23002FD1
:107C000001DA7F422D230A21021EA0F1010000DCCF
:107C10005FB197FBF1FC97FBF1F201FB1C7C17466F
:107C20000CF1300C08F801CDEEE7A8F1010003706B
:107C30002188090501D5452100E06521A0F1010851
:107C400000F8011C09980FA9A1EB0807FF1D00B15E
:107C50000120411901EBEA70A1693844081A401E5D
:107C6000A0612078C00602D42046AFF300800998B6
:107C700028B1D4E901219047206A401C2062207875
:107C8000C00622D52046AFF300801EE0002E04DBA4
:107C9000B34502DD01A8805D00E03020D4E9012178
:107CA0009047206A401C2062761CAAF101005FEA1E
:107CB000000A0AD100F032F8C0680168405CD4E9DB
:107CC00001219047206A401C2062281EA5F1010571
:107CD000DCDC07E0D4E9012118F8010B9047206AA9
:107CE000401C2062381EA7F10107F3DC2046AFF3E9
:107CF0000080032011B043E6074B70B50D467B446E
:107D000000F05FF80446284600F01CF910B14FF06F
:107D1000FF3070BD204670BD67D3FFFF004870473D
:107D20003C090020004870471C09002030B5B0F124
:107D30000A024FEA900E71F100034EEA817EB0EB29
:107D40000E0061EB91014FEA101E4EEA017E10EB2E
:107D50000E0041EB11114FEA102E4EEA016E10EBAE
:107D60000E0041EB11214FEA104E4EEA014E10EB8E
:107D70000E0041EB1141401841F100014FEAD000E3
:107D800040EA41704FEAD10110EB80054FEA8104CF
:107D900044EA907444EB01046D1944EB0404521B53
:107DA000A3414FF0000348BF0A3200D530BD401C4C
:107DB00041F1000130BD000001694A1C02610878F0
:107DC000704700B58FB0CDE901310021059105491B
:107DD0007944CDE9031011466846FFF7D9FB0FB08F
:107DE00000BD0000E5FFFFFF2DE9F0411F460446FE
:107DF00003260168072A01F4006004DB08B116A518
:107E000005E016A503E008B115A500E015A521F0D1
:107E100010002060A069C01EA0610FB1401EA061CB
:107E20002046AFF300804FB1D4E901213846904796
:107E3000206A401C2062C01C206206E0206AFAE72B
:107E4000D4E9012115F8010B9047761EF8D220469F
:107E5000AFF30080BDE8F0814E414E006E616E00D0
:107E6000494E4600696E66002DE9F0478146164688
:107E70008AB0334878440DC88DE80D003048784406
:107E8000801C03AC0DC884E80D0041F69B3008440B
:107E9000372190FBF1F290FBF1F5A5F1800501FB94
:107EA00012041B3C02D56442012000E00020DFF8F0
:107EB00090A080460027FA44AAF1BE0A0DE0E00730
:107EC00009D03246684607EB47010AEB810100F012
:107ED00034FB8DE8070064107F1C002CEFD1184F95
:107EE0007F44AC3F18E0E80714D007EB04100DF115
:107EF000180A90E80E008AE80E00C068F04201D12E
:107F000098190890324606A903A800F016FB03ABA7
:107F100083E807006D10641C002DE4D132466946E9
:107F2000B8F1000F03A802D000F0F3FA01E000F06E
:107F300004FBC9E90001C9F808200AB0BDE8F087D0
:107F400054260000007B00F0800070470048704716
:107F50001C0900207546FFF7F9FFAE46050069468B
:107F6000534620F00700854618B020B5FAF7A8FD63
:107F7000BDE820404FF000064FF000074FF000082A
:107F80004FF0000B21F00701AC46ACE8C009ACE8AB
:107F9000C009ACE8C009ACE8C0098D46704710B50F
:107FA0000446AFF300802046BDE81040F8F718B94A
:107FB0004FF0013C50F8042B51F8043B9A4221D178
:107FC000A2EB0C03934313EACC1317D150F8042B04
:107FD00051F8043B9A4215D1A2EB0C03934313EAE8
:107FE000CC130BD150F8042B51F8043B9A4209D121
:107FF000A2EB0C03934313EACC13DBD04FF0000049
:10800000704700BFD01A01BAB1FA81F101F018012E
:1080100022FA01F0CB40C1F12001DBB2C0B2C01A9C
:108020002CFA01F3D11A914311EAC311E6D170473A
:108030005FEA400C08BF91F0000F4FEA8C234FEA33
:10804000C12243EA51514FEA1C5018BF00F5F040DD
:108050004FEA300018BF41F000415FEA6C5C00F06D
:108060002980BCF1FF3F08BF40F080407047130CEF
:1080700006BF12044FF0100C4FF0000C130E04BF9B
:1080800012020CF1080C130F04BF12010CF1040CC6
:10809000930F04BF92000CF1020CD30F04BF5200E7
:1080A0000CF1010C11464FF00002A0F11F00A0EBF3
:1080B0000C00704711F0004F08BF704731F00041CD
:1080C0003FF4D5AF0B0C06BF09044FF0100C4FF076
:1080D000000C0B0E04BF09020CF1080C0B0F04BFBF
:1080E00009010CF1040C8B0F04BF89000CF1020C88
:1080F000CB0F04BF49000CF1010CCCF12003A0EB25
:108100000C0022FA03F302FA0CF241EA030100F137
:108110000100704720F07F4C80EA030023F07F4786
:10812000ACEB070303F57C5300F0004003F1FF03C1
:108130002DE980494FEA154B09B44FEA144325EA6B
:108140000B4E24EA03480FF2042606EB13274908D6
:108150003E785FEA320203FB0667C7F5000707FBBC
:1081600006F64FEA54374FEAD64606F1020607FBF9
:10817000066CCCF1005C4FEA1C472CEA074C07FB6D
:1081800006F40CFB06F504EB15464FEA961634BFD1
:1081900000204FF000404FEAD13706FB07FC4FEAC2
:1081A0001C4C0CFB0BF7D21B03FB0CF761EB07011C
:1081B0000CFB0EF7B0EB074072EB17420CFB08F715
:1081C00034BFA2EB0742B2EB074261EB17414FEA23
:1081D0000C444FEA910706FB07FC4FEA1C4C0CFBD2
:1081E0000BF7B0EBC74072EB573203FB0CF734BF11
:1081F000A2EBC742B2EBC74261EB57310CFB0EF763
:10820000B0EBC70072EB57720CFB08F734BFA2EB60
:10821000C702B2EBC70261EB5771039F4FEA81615E
:1082200041EA921104EBCC044FEAD1374FEA826263
:1082300006FB07FC42EA90124FEA80604FEA1C4CB2
:108240000CFB0BF7D21B03FB0CF761EB07010CFBDC
:108250000EF7B0EB074072EB17420CFB08F734BF88
:10826000A2EB0742B2EB074261EB17414FEA8C5594
:108270004FEA910704EB9C2406FB07FC4FEA1C4CD9
:108280000CFB0BF7B0EBC74072EB573203FB0CF75C
:1082900034BFA2EBC742B2EBC74261EB57310CFBD4
:1082A0000EF7B0EBC70072EB57720CFB08F734BF48
:1082B000A2EBC702B2EBC70261EB577115EB4C257D
:1082C0004FEA816141EA92114FEA82624FEAD13767
:1082D00042EA901206FB07FC44F100044FEA80607A
:1082E0004FEA1C4C0CFB0BF7D21B03FB0CF761EBAA
:1082F00007010CFB0EF7B0EB074072EB17420CFBCB
:1083000008F734BFA2EB0742B2EB074261EB17411B
:1083100015EB1C154FEA813141EA92414FEA823256
:1083200042EA90424FEA80304FEA0C7644F1000472
:1083300048EA03434EEA0B484FF0000EB2EB080C3C
:1083400071EB030724BF624639464EEB0E0E4FF029
:10835000000B0018524149414BEB0B0BB2EB080CE0
:1083600071EB03077BF1000B24BF624639464EEBED
:108370000E0E4FF0000B0018524149414BEB0B0B16
:10838000B2EB080C71EB03077BF1000B24BF6246D4
:1083900039464EEB0E0E51EA020718BF46F00106B1
:1083A00016EB0E7655F1000254F1000103D5BDE83D
:1083B0008901BDE80088BDE88901BDE80048B6191B
:1083C000524141EB0101A3F10103704780807F7EA0
:1083D0007D7C7B7A7978777676757473727171703B
:1083E0006F6E6E6D6C6C6B6A6A69686867666665ED
:1083F0006464636362616160605F5F5E5E5D5D5C7B
:108400005C5B5B5A5A5959585857575656555555EB
:108410005454535352525251515050504F4F4F4E4B
:108420004E4D4D4D4C4C4C4B4B4B4A4A4A49494999
:1084300048484847474747464646454545444444DB
:10844000444343434342424242414141002B26D4EC
:10845000770021D01CB54FEA370703B44FF0100066
:108460004FF010014FF000000FBCBDE810400BF1C1
:10847000010BBBF1010F08BF5FEA170722BF12F122
:10848000010211F101014FF0004143F1000300F03E
:10849000004043EA00007047F9D35708DAE746EA9C
:1084A000064613F1400F4FEA16461FDD13F1200F69
:1084B000DFBF16430A46002120335B42C8D0C3F118
:1084C000200746EA064602FA07F74FEA164646EA4A
:1084D0000706C3F1200722FA03F201FA07F721FA8F
:1084E00003F14FF0000342EA0702B1E746EA020651
:1084F00046EA06464FEA164646EA0106BCBF46EA89
:108500000646360C4FF000034FF000024FF000011A
:108510009EE72DE9C048934630B491E8380007C87B
:1085200031EA400C48BF34EA430C03D5FFF7F2FDB3
:10853000FFF78CFFF0BCBDE800882DE9C0489346EA
:1085400030B491E8380007C810F0804F08BF13F02E
:10855000804F03D100F005F8FFF778FFF0BCBDE8CD
:10856000008820F07F4780EA030023F07F4C07EB70
:108570000C03A3F57C5300F00040A3F1FE0392F03E
:10858000000F00F0B38095F0000F00F077802DE928
:1085900001494FEA11404FEA144621EA004800FB26
:1085A00006FC24EA064708FB06F607FB08F800FB72
:1085B00007F718EB06484CEB164C4FEA124B18EB3A
:1085C00007484FEA15464CEB174022EA0B4E0BFBCF
:1085D00006FC25EA06470EFB06F607FB0EFE0BFB24
:1085E00007F71EEB064E4CEB164C4FF000061EEB49
:1085F000074E4CEB174B18EB0B0840F1000018EB43
:108600000E0B58EB000840F100008F1A4FF00001EC
:108610003CBFC943661B14BFB5EB040C00213CBF33
:10862000C943F61B4FEA17444EEA8E0E27EA04456B
:108630004FEA1C4704FB07622CEA074C05FB07F7CF
:108640000CFB05F604FB0CFC16EB074642EB17424D
:1086500016EB0C4642EB1C421BEB060658EB0202E3
:10866000414146EA9E0601D5BDE80189B61952414D
:1086700041EB0101A3F10103BDE801894FEA144573
:108680004FEA114724EA054621EA074C05FB07F4A7
:1086900006FB07F70CFB06F105FB0CFC11EB074191
:1086A00044EB17444FEA124711EB0C4144EB1C44D6
:1086B00022EA074C05FB07F206FB07F70CFB06F660
:1086C00005FB0CFC16EB074642EB174216EB0C467B
:1086D00042EB1C456A1854F1000148BF7047B619B7
:1086E000524141EB0101A3F10103704795F0000FE6
:1086F00037D04FEA11424FEA144721EA024624EAF2
:10870000074C02FB07F106FB07F70CFB06F402FB24
:108710000CFC14EB074441EB17414FEA154714EBEF
:108720000C4441EB1C4125EA074C02FB07F506FB14
:1087300007F70CFB06F602FB0CFC16EB074645EBB5
:10874000174516EB0C4645EB1C42121951F100017E
:1087500048BF7047B619524141EB0101A3F1010333
:1087600070474FEA14454FEA114724EA054621EACB
:10877000074C05FB07F106FB07F70CFB06F24FF071
:10878000000605FB0CFC12EB074241EB174112EB14
:108790000C4251EB1C4148BF7047921841EB01015C
:1087A000A3F101037047490050EAC12018BF04201B
:1087B0004A0D18BF40F0010040F2FF72B2EB515F6A
:1087C00008BF40F00200012808BF052070470000E4
:1087D0002DE9F74F144694B00021C4E90211159910
:1087E000079121F00045C9498D4206DC1599C4E97D
:1087F000000117B00020BDE8F08FC549DFF814A3D1
:10880000A9423CDD0799C44E0029C44FC44A1599BA
:10881000534619DD01F020F8554506D0C14AC24B38
:1088200001F01AF8C4E900010AE04FF0D352BE4B40
:1088300001F012F832463B4601F00EF8C4E900019F
:1088400017B00120BDE8F08F00F0C2FB554506D0FF
:10885000B44AB54B00F0BCFBC4E900010AE04FF09C
:10886000D352B14B00F0B4FB32463B4600F0B0FBB4
:10887000C4E9000117B04FF0FF30BDE8F08FAB49FD
:10888000A942159978DB21F0004183468846A84A21
:10889000A84B00F047FE0022A74B00F099FB00F028
:1088A000ABFD099000F0D7FD06460F469C4A5346A3
:1088B00000F038FE43465A4600F0C2FF80468A4622
:1088C000984A994B3046394600F02CFE2A0D012576
:1088D0000B924246534600F0B3FF032DC4E900015A
:1088E00039D00B98C1F30A51401A05EB45111139E3
:1088F000814230DA9148C346784400EB0510CDF848
:108900000CA00C90D0E900233046394600F00AFE56
:1089100002460B46049106905846039900F09CFFCE
:1089200080468A4602460B465846039900F094FF5B
:10893000049B069A00F090FF83460C9803913946F9
:10894000D0E90223304600F0EDFD5A46039B00F0CB
:1089500083FF6D1CBDE707980028A2BF099817B0D8
:10896000BDE8F08F616881F000416160099817B03F
:108970004042BDE8F08FFFE784461598C1F313012C
:10898000C0F30A50A0F2F5304FEA601800F01F065D
:10899000C6F12000139000200690079041F4801E3D
:1089A00005206D4676B1664A08EB00017A4452F81C
:1089B000213002EB8101B3404A68139922FA01F198
:1089C000194305E05F4908EB0002794451F8221091
:1089D000A1FB0E27A1FB0C131A449A4234BF0123BA
:1089E000002303EB070A05EB8003D3E901B70F442B
:1089F0008F4234BF0121002193448B4411B1934530
:108A000002D903E0934501D2012100E00021C3E92E
:108A100001B7514445F82010011EA0F10100C1DC4E
:108A20000298059F00F10050800F12900298DDE936
:108A30000356800000F00FFD834628460D9100F09C
:108A400021FD6FF01D0201F0FEFACDE90E01304666
:108A500000F018FD6FF03D0201F0F5FA80468A46FD
:108A6000384600F00FFD6FF05D0201F0ECFA0746AA
:108A700042465346119100F0ABFADDE90E2300F0B7
:108A8000A7FA5A460D9B00F0A3FA00250E465A4657
:108A900028460D9B00F0E0FEDDE90E2300F0DCFE31
:108AA0004246534600F0D8FE3A46119B00F0C8FEFD
:108AB000DFF898A0244A534600F034FD0746884664
:108AC000234A244B3146284600F02CFD3A464346C3
:108AD00000F07EFA074688464FF0A84253463146DA
:108AE000284600F01FFD3A46434600F071FA159AF9
:108AF00012F0004F04D0129A81F0004152421292BB
:108B0000C4E90001129817B0BDE8F08FFB21E93FDE
:108B10007CD90240FB21F93F7370032E8A19A33BD5
:108B2000000040543163621A61B4D03DFB213941E9
:108B300083C8C96D305FE43F0000E03F641A000065
:108B4000E0190000C2190000182D4454FB21F93D22
:108B50003326A611460B113C2DE9FF4D21F00048AC
:108B600007460C46B8F1795F08DA00F045FC0028AA
:108B700001BF0020324904B0BDE8F08D3A462346DB
:108B80001046194600F0CEFC054602462D480E461A
:108B90000B460621784400F05DF82A46334600F083
:108BA000C1FCDDE9022382468B463846214600F0AF
:108BB000B9FC04460F4652465B462846314600F053
:108BC000B1FC22463B4600F047FE07468A464FF07E
:108BD000FF322846314601F036FA1B4A90450ADA40
:108BE0003A46534600F038FE04B00022BDE8F04D8E
:108BF000134B00F025BE154A4245A8BFA8F5001545
:108C00004FF00004B8BF124D22462B4600F024FE60
:108C10000646884622462B460020094900F01CFEE5
:108C200004460D463A4653463046414600F014FE8F
:108C300004B022462B46BDE8F04D00F001BE000016
:108C40000000F03F981700003333D33F0000E93FA6
:108C50000000D23F2DE9F0414F1E00EBC701044652
:108C6000D1E9000115461E4637F006020DD02A460E
:108C7000334600F057FC7F1E04EBC703D3E9002303
:108C800000F0A6F937F00602F1D1022F25D0042F0B
:108C900013D0062F18BFBDE8F0812A46334600F0F6
:108CA00041FCD4E90A2300F093F92A46334600F048
:108CB00039FCD4E9082300F08BF92A46334600F04A
:108CC00031FCD4E9062300F083F92A46334600F04C
:108CD00029FCD4E9042300F07BF92A46334600F04E
:108CE00021FCD4E9022300F073F92A46334600F050
:108CF00019FCD4E90023BDE8F04100F069B9000097
:108D00002DE9FF4D054621F0004084B00C46B0F13E
:108D1000795F0BDA2846FFF746FD042808BF00F00C
:108D20006FF8284608B02146BDE8F08D2A460B466C
:108D3000104600F0F7FB06460F462A46234600F091
:108D4000F1FB804626488A4632463B460521784458
:108D5000FFF780FF83461098029160B3214A224BAF
:108D60004046514600F0DEFBCDE900015A46404640
:108D70005146029B00F0D6FB82468846DDE906019B
:108D80004FF0FF3201F05FF95246434600F064FDB8
:108D900032463B4600F0C6FBDDE9062300F05CFDF1
:108DA000DDE9002300F058FD08B02A462346BDE85F
:108DB000F04D00F045BD0B465A463046394600F0AE
:108DC000B1FB084A084B00F003F94246534600F055
:108DD000A9FB08B02A462346BDE8F04D00F0F8B8DC
:108DE000D6160000495555555555C5BF012201F00D
:108DF0002AB9002213461046114600F0A5B900001A
:108E0000024A0020110701F01EB9000001FDFFFF1A
:108E100000B5244B21F0004287B09A42DCBF00220B
:108E2000134629DD204B9A4208D140B94FF001008A
:108E3000FEF7F6FCFFF7DDFF07B000BD03DBFFF731
:108E4000D5FF07B000BD02AAFFF7C2FC10F0030176
:108E500004BF0DF1080C9CE80F000DD00120012982
:108E60000ED0022914D00DF1080C00909CE80F00E0
:108E7000FFF746FF07B000BDFFF76EFE07B000BD6D
:108E80000DF1080C00909CE80F00FFF739FF05E09A
:108E90000DF1080C9CE80F00FFF75EFE07B081F0B3
:108EA000004100BDFB21E93F0000F07F2DE9F04DBE
:108EB00007460E4600F06AFC04460D463A46334625
:108EC00000F0BEFCDFF86CA0DFF86CB01B4B07466F
:108ED000884616F0004F4FF000020AD000F0E6FA84
:108EE0000AD900225B463846414600F019FC1BD2E5
:108EF00012E000F0DBFA08D2002253462046294651
:108F000000F0AAFC04460D460EE000225B463846FF
:108F1000414600F005FC07D800225346204629466A
:108F200000F056F804460D463146204665F31E0112
:108F3000BDE8F08D0000F03F0000E03F0000E0BF22
:108F400010B500290AD00878002807D005487844D1
:108F5000FFF72EF8002801D0002010BD0248784409
:108F600010BD0000B6150000AE15000021F0004253
:108F7000A2F16052B2F5801F01F0004328BFD2F188
:108F80007F6C0BD95FEA001C43EAC20242EB5070CF
:108F900018BF704728BF20F001007047B2F5801F4E
:108FA000BCBF184670474FEA410C1CF5001F02D2A7
:108FB000084600F09ABF70B500F05EFB0000008923
:108FC000FFF7F6BF4FF00040A0F5800070470000AB
:108FD00010B591EA030F48BF83F0004300F14484C9
:108FE000841A71EB030C05D2121943EB0C03001B1E
:108FF00061EB0C01DFF824E14FEA1154A4EB135CA0
:109000001EEA430F18BF9EEA445F73D023EA0E03A3
:10901000DCF1200E21EA045143F4801332D322FA0A
:109020000CFE10EB0E0023FA0CFE41EB0E01CCF10E
:10903000200E03FA0EFE10EB0E0051F10001B1F507
:10904000801FCCF1200E32D201EB045112FA0EF245
:10905000BDE8104058BF7047401C38BF5FEA42026D
:1090600018BF7047002814BF20F0010041F1000133
:109070004FEA410313F5001F38BF7047A1F1C0410B
:1090800000F048BB012A43EB0302ACF1200CDCF1F9
:109090001F0E32BF4FF0000E23FA0CF310EB03004B
:1090A00041EB0451B4EB115FD0D0A1EB045101F5B9
:1090B000801149085FEA300001EB04510ED350F1F2
:1090C000000038BF12FA0EFE08D1BDE81040C9E713
:1090D000401C38BF5FEA4202CAD1C3E7BDE8104076
:1090E0004FEA410313F5001F38BF7047A1F1C0419B
:1090F00000F010BB9EEA445F08D011EA5E0FBDE8A5
:10910000104004BF01F0004100207047BDE810404E
:1091100070B500F0B1FA00BF64FBBE3E0000E0FF96
:1091200002494FF0000000F05CBF00BF0000F87F74
:10913000491058BFC1F140415B1058BFC3F14043D3
:109140008B42EFF3008070472DE9C04130B4DFF867
:10915000A0C23CEA111418BF3CEA131400F0EC80E2
:1091600081EA03051CEA111444EAD57418BF1CEA0D
:10917000131500F0C780A4EB05044FF0004545EA45
:10918000C12145EAC32341EA505143EA525304F155
:109190007F74994204F500344FEAC0204FEAC2229E
:1091A00008BF904200F09C804FEA13650FF2401612
:1091B000765D4FEA134506FB05F7C7F1807706FB9E
:1091C00007F74FEAD737A7FB03687642C8F5803820
:1091D000A7FB06CE38BFA8F1010807FB08E64FF051
:1091E000000EA6FB028CE6FB03CEDCF1000CCEF1F8
:1091F000004E38BFAEF1010EA6FB0C584FF0000731
:109200004FF00005E6FB0E87A1FB08C6A0FB07CECA
:1092100016EB0E0645F10005E1FB076515F1E04E82
:109220007EBFA4F580345FEA46066D4116F18007E3
:1092300045F100054FEA17274FEA066647EA05673A
:10924000A6F1DE46B6F1805F4FEA15251FD93846F4
:1092500024F0010C05EBC471BCF1FE6F01EB0C11A5
:1092600002D8F0BCBDE8008124425CBF01F5801E3D
:109270009EEAC47F02D4F0BCBDE80081244238D409
:10928000F0BCA1F1C041BDE8004100F043BA4FEA93
:10929000D22242EA43524FEAD323A7FB02864FEA87
:1092A000D02040EA415007FB03661EEA0E0F4FEA4A
:1092B000D12105FB026658BFA6EB0056B6EB00565F
:1092C0004FEA520E4EEAC37E18EB0E0E56EB530ECB
:1092D000BDD518EB02085E417F1C55F10005B6E7CD
:1092E0004FF480154FF000074FF000064FF00008D4
:1092F000ADE7F0BC4FF0000001F1C04101F00041CA
:10930000BDE8008111EA0C1F0CEA131500D00CE037
:1093100013EA0C1F00F025804FF00000F0BC81EA3A
:10932000030101F00041BDE80081F0BCBDE800414F
:1093300081EA030100F0EEB9F0BCBDE8004170B570
:1093400000F09AF9097EFC3E00F007B881EA0301BB
:109350004FF0000001F00041704781EA030100F086
:10936000D9B9F0BCBDE800414FF000002149704779
:10937000FFFDFBF9F7F5F4F2F0EEEDEBE9E8E6E4DA
:10938000E3E1E0DEDDDBDAD8D7D5D4D3D1D0CFCD61
:10939000CCCBCAC8C7C6C5C4C2C1C0BFBEBDBCBB9A
:1093A000BAB9B8B7B6B5B4B3B2B1B0AFAEADACAB95
:1093B000AAA9A8A8A7A6A5A4A3A3A2A1A09F9F9E6F
:1093C0009D9C9C9B9A999998979796959594939321
:1093D000929191908F8F8E8E8D8C8C8B8B8A8989B8
:1093E000888887878685858484838382828181803B
:1093F0000000FF070000F87F4FEA41034FEA535394
:10940000A3F58063D3F11E03C8BFD3F1210C0CDD9B
:109410004FF0004242EAC12242EA505232FA03FCC3
:109420008CEAE17CACEBE1707047102BC4BF0020EC
:10943000704703F5787CBCF1FF3F04D06FF0004229
:1094400082EA2100704770B500F016F94992248035
:1094500000207047F2E710F0004248BF4042B0FAE7
:1094600080F310FA03F10AD0C3F11D0303F5806302
:109470004FEA415002EB035202EBD12170474FF00B
:1094800000007047B0FA80F310FA03F10AD0C3F17C
:109490001D0303F580634FEA41504FEA035202EB8C
:1094A000D12170474FF000007047000051EA030CD3
:1094B00017D41CF5801F58BFBCF5801F00F1068033
:1094C000994218BF704708BF9042704707D711F5FF
:1094D000801F58BF13F5801F19D4994270478942E5
:1094E00070471CF5801F08D5BCF5801FF7D58B424F
:1094F00018BF704708BF824270474FF4001C1CEB36
:10950000410F38BF1CEB430F01D28B42704770B53F
:1095100000F0B2F8922449004FF000514FF0805310
:10952000FFF706BEDFF848C170B51CEA111E1EBF6A
:109530001CEA13159EEA0C0F95EA0C0F00F06F80E1
:1095400081EA030423EA4C134EEAD47E21EA4C114B
:1095500041F4801143F48013AE44A1FB024CA0FB04
:109560000365AEF17F7E361955EB0C05A1FB034C6C
:109570004CF10003A0FB021C16EB0C06654153F1F5
:109580000003094218BF46F0010613F4007F0BD117
:109590004FEA03314FEA0530340341EA155140EAFE
:1095A00016506FF003020AE04FEAC3214FEAC520CC
:1095B000F40241EA555140EA56506FF0020202EBC4
:1095C0002E4201EB025585EACE710AD05FEA440CC7
:1095D00018BF24F0004450F1000041F1000120EADE
:1095E000D47040F2FE7C624500D270BDA84214BF28
:1095F0004FF080444FF04044002E08BF0024BEF1DD
:10960000806FA8BFA1F1C041BDE8704080F28280A8
:109610004FF0000001F1C04101F0004170479EEAA7
:109620000C0F0CEA131518BF95EA0C0F06D04FF07B
:10963000000081EA030E0EF0004170BD00F01CF83E
:109640008900013E00F007B800F009B84FEA430C6A
:109650005FEA5C5C08D081EA030100F05BB84FEA86
:10966000410C5FEA5C5CF6D14FF0000001497047A5
:109670000000FF070000F87F0EF1020E2EF0030E2F
:109680005EF8046B364205D4012A43EB030515F559
:10969000001F12D8012841EB010C1CF5001F0CD84B
:1096A0000ED14FEAD17C15F5001F0CEB4C0C0CF1E0
:1096B000020C08BF4CEBD37C04E04FF0080C01E037
:1096C0004FEAD37C0CEB4C0526FA05F606F00706AC
:1096D000B6F1040C06D20EEB860CBDE870404CF0DF
:1096E000010C6047DFE80CF0090B02024FF000416B
:1096F0004FF00000A1F5002170BD19461046012869
:1097000051EB010418BFD4F5001484BF002001F010
:10971000004170BD0808A0F500114FEA3101704703
:1097200053EA010C17D41CF5801F58BFBCF5801FED
:1097300000F106808B4218BF704708BF8242704715
:1097400007D713F5801F58BF11F5801F19D48B421E
:1097500070479B4270471CF5801F08D5BCF5801FE1
:10976000F7D5994218BF704708BF904270474FF431
:10977000001C1CEB430F38BF1CEB410F01D2994278
:1097800070470FB40CBC03BCFFF7C1BE5FEA410CCD
:109790005FEA5C5CACF580635B1C39D4D3F13402C6
:1097A00040F34580B2F1200314DA4FF0010C0CFABB
:1097B00002FCACF101030340B3EB5C0220EA0300BE
:1097C00008BF10EA0C0F98BF704710EB0C0041F176
:1097D000000170470AD0C3F1200201FA02FC0128FF
:1097E00021FA03F101FA03F14CF100004FF0010CF2
:1097F0000CFA03FCACF10103B0F1004F21EA0301C4
:1098000008BF11EA0C0F4FF0000088BF6144704799
:10981000B3F1FF3F28BF50EAC12C01F000414FF0E7
:10982000000084BF41F07C5141F470017047B3F5F2
:10983000806FB8BF704770B5FFF71EFF40DBB6BE44
:1098400091EA030F10B581F000413FF5C9AB83F0F9
:10985000004300F009B8000010B591EA030F48BFBB
:1098600083F000433FF5BCAB841A71EB030C07D2C5
:1098700012198CF0004C43EB0C03001B61EB0C0144
:10988000DFF8A4E14FEA1154A4EB135C1EEA430F86
:1098900018BF9EEA445F00F0B08023EA6E03524294
:1098A00021EA0451C3EB6E0338BF5B1EDCF1200ECE
:1098B00025D322FA0CFE10EB0E0043FA0CFE41EB0E
:1098C0000E01CCF1200E03FA0EFE10EB0E0051F14A
:1098D0000001CCF1200E29D412FA0EF201EB045152
:1098E000BDE8104058BF7047401C1CBFB2F1004F8C
:1098F000704700280CBF491C20F00100704712EB94
:10990000020E43EB030218BF4FF0010E4EEA420273
:10991000ACF1200CDCF11E0E54D943FA0CFE10EB16
:109920000E0051F1FF31CCF11E0ED5D50EF1010E16
:1099300012FA0EFE404141EB010101EB445C5FEA8B
:109940005C5C10D910EBDE7001EB045138BFBEF146
:10995000004FBDE8104018BF704700280CBF491CDD
:1099600020F00100704730D24FEAD42C11F50011DD
:1099700024F400641BD0B1FA81F20B3AA41AA41E9D
:10998000D2F12003914030FA03F31943904001EBE8
:10999000CC71002C01EB0451BDE81040A8BF70470A
:1099A00001F1C0414FF0000001F000417047B0FAF2
:1099B00080F310FA03F100D110BDE41A173C4805FA
:1099C000C90AE4E701EB045110BD491001EB045151
:1099D000BDE810404FEA300002E04FF00001704750
:1099E0004A0008BF0042F8D0B2F5001F28BF7047F8
:1099F00001F000414FF0000070479EEA445F07D03D
:109A000011EA5E0FBDE8104004BF0021002070473E
:109A1000BDE8104070B5FFF72FFE00BF40DFF63EF7
:109A200083F00041104670470000E0FF43004FEA1A
:109A3000D30C4FEA3C0C43401FBF40070CF1605170
:109A400013F0FE4F70471CF0006F03D100200CF0A4
:109A5000004170470CF0004343EA507010B540EAF3
:109A6000CC0000F0FCF900BF000000924FEA0001BA
:109A7000FFF750BE4FF000414FF00000A1F500216C
:109A80007047000090EA010F48BF81F0004100F1EB
:109A90003882421A3CBF801A89184FEAD0524FF0E0
:109AA0007F4C1CEA410FA2EBD15318BF9CEA026F16
:109AB00000F03B804FF0004C4CEA00204CEA0121C2
:109AC00021FA03FC10EB0C0C1ED202F1FF325FEA0C
:109AD0001C2040EBC25038BF70471CF07F0F4FEA8C
:109AE000400C18BFBCF17F4F38BF7047C3F1200353
:109AF000994008BF20F00100BCF17F4F38BF70478C
:109B0000A0F1C04000F0F1B94FEA3C00000A40EB80
:109B1000C25028BF1CF0FF0F4FEA400CE6D018BF20
:109B2000BCF17F4F38BF7047EAE79CEA026F05D06F
:109B300010EA5C0F08BF00F00040704710B500F05D
:109B40008EF900BF64FBBE3E4FF47F0C1CEAD012BE
:109B50001EBF1CEAD11392EA0C0F93EA0C0F00F01F
:109B6000858090EA010F48BF42F4807240F4000CF7
:109B700041F400002CF07F4120F07F4000B581428D
:109B8000A2EB03020FF2081CACEB504EC0F1000038
:109B90009EF800E04FEA4E0E00FB0EFC38BF490075
:109BA0004FEA2C1C02F5FA020CFB0EF34FEACE1E14
:109BB0004FEA112C4FEAC1210EEB635E42EB2242C9
:109BC0000EFB0CFC4FEA1C5300FB03114FEA112C57
:109BD0004FEA01310EFB0CFC4FEADC4C00FB0C1190
:109BE000C14228BF09184CEB03335DF804EB10EBBE
:109BF000410143EBC250B2F57C0F38BF704729D505
:109C000012F0F00F1CBF00F1C04000F000407047A0
:109C1000008182838485868788898B8C8D8E8F9145
:109C20009293959697999A9C9D9FA0A2A3A5A7A869
:109C3000AAACAEB0B2B3B5B7B9BCBEC0C2C5C7C995
:109C4000CCCED1D4D7D9DCDFE2E6E9ECF0F3F7FAF9
:109C5000FE0000004FEA400C0CF1807CBCF17E4F0E
:109C600028BF7047B0F1C04000F03FB990EA010F43
:109C70000CEAD11348BF42F48072624538BF634595
:109C800007D213F47F0F16D080EA010000F00040E5
:109C9000704710B500F0E3F8097EFC3E00F005B80F
:109CA00080EA010000F00040704780EA010000F007
:109CB000004000F01AB912F47F0F04BF0248704749
:109CC00080EA010000F011B90000C07F41000B0ED6
:109CD000D3F19E0208D950F400034FEA032323FA7C
:109CE00002F048BF4042704710B500F0B8F800BF1E
:109CF00049922480002070476FF0004282EA2000E1
:109D00007047000010F0004148BF4042B0FA80F3B5
:109D100010FA03F2C3F19D030BD051EAC35101EBDA
:109D20001220530638BF704700F1010008BF20F031
:109D300001007047B0FA80F310FA03F2C3F19D03FB
:109D40000AD0D90501EB1220530638BF704700F145
:109D5000010008BF20F00100704700004FF47F0CA5
:109D60001CEAD0121EBF1CEAD11392EA0C0F93EA30
:109D70000C0F00F0478090EA010F48BF42F4807258
:109D80004FF0004C4CEA00204CEA012102EB0302A8
:109D9000A0FB0113A2F50002002918BF43F0010344
:109DA0005B0028BF4FEA330342EB22425FEA132CE9
:109DB0004CEBC2502EBFBCEB436FB2F57C0F70472B
:109DC0004FEA036CBCF1004F08BF20F00100B2F570
:109DD0007C0F38BF70470BD582F0FF0212F5803F31
:109DE000C8BF704700F1C040D8BF00F000407047C6
:109DF00000F5000C5FEA4C0C48BF7047B0F1C04062
:109E000000F073B890EA010F0CEAD11348BF42F496
:109E10008072624538BF634504D280EA010000F0D9
:109E20000040704710B500F01AF800BF8900013EED
:109E300000F007B800F009B85FEA410C5FEA1C6C5B
:109E400008D080EA010000F050B85FEA400C5FEAF9
:109E50001C6CF6D14FF00040A0F5800070470EF169
:109E6000020E2EF0030E5EF8044B244204D44FEA97
:109E70004102B2F17F4F11D84FEA4003B3F17F4F57
:109E80000CD80ED14FEAD07CB2F17F4F0CEB4C0CCA
:109E90000CF1020C08BF4CEBD17C04E04FF0080C35
:109EA00001E04FEAD17C0CEB4C0324FA03F404F0FC
:109EB0000704B4F1040C06D20EEB840CBDE810408C
:109EC0004CF0010C6047DFE80CF0070802024FF08D
:109ED0000040A0F5800010BD0846420018BFD2F136
:109EE000807288BF00F0004010BDFF2141EAD050D1
:109EF000C005704790EA010F48BF81F000413FF56F
:109F0000C8AD421A04D882F00042A0EB020011440E
:109F10004FEAD0524FF07F4C1CEA410FA2EBD153D5
:109F200018BF9CEA026F4AD04FF0004C4CEA002068
:109F30004CEA012121FA03FCB0EB0C0C0FD412F017
:109F4000FE0F36D05FEA4C001DD5001240EBC25028
:109F500038BF70471CF03F0F18BF70470BE0A2F1ED
:109F600001025FEA1C2040EBC25038BF70471CF072
:109F70007F0F18BF7047C3F12003994014BF401EE4
:109F800020F00100704780084FEA122308BF704795
:109F9000B0FA80FCA2EB0C02CCF1280C60FA0CF0B9
:109FA00093EA122F04BF00EBC25070474FEAC37010
:109FB0007047130A5FEADC1008BF7047F6E79CEAB7
:109FC000026F04D010EA5C0F08BF0020704710B584
:109FD000FFF745FF40DFF63E81F000407047FDF798
:109FE00055BD0CF00F03092B08BF082000F0598065
:109FF0000A2B0BD0082B18BF704708BF1CF0400F6E
:10A000000AD04FF000004FF0000170471CF0400FE5
:10A0100018BF4FF0004070471CF0100F08D020F020
:10A02000704300F07F4242EAD3014FEA4370704729
:10A0300000F0604021F07F4242EA000201F07F40E0
:10A0400040EA727070474FF0FF0C4CF4E06C1CEA71
:10A0500011531CBF9CEA030C9445C2BFDA4201EBCA
:10A0600002517047002B0DD0BCF1000F0FD0002A19
:10A0700001F00041A4BF41F0E04141F07F614FF0A9
:10A080000000704701F000414FF00000704750EAB7
:10A0900001334FF09B0C18BF4CF0806C7FF440A84C
:10A0A00070471CF4801F11D01CF4E02F03D06FEA1E
:10A0B000CC31490070474FF04050EFF3008222F05E
:10A0C000704242EA000282F3008870474FF00000BD
:10A0D0007047120100020000004033280200020213
:10A0E0000102030109022200010100A0320904005B
:10A0F00000010300000009211001000122AF010747
:10A1000005810340000105030905A1010600FF09BF
:10A1100001A10205018501093B150026FF00750814
:10A1200095018103093B150027FFFF00007510957D
:10A13000018103093B150027FFFF00007510950101
:10A140008103093B150027FFFF0000751095018171
:10A1500003093B150026FF00750895108103093B94
:10A16000150026FF00750895108103093B15002690
:10A17000FF00750895108103093B150027FFFF00BC
:10A18000007510950381038502093B150027FFFF29
:10A19000000075109501B103093B150026FF0075FD
:10A1A000089504B1038503093B150027FFFF000054
:10A1B00075109501B103093B150026FF0075089540
:10A1C00042B1038504093B150027FFFF000075100D
:10A1D0009501B103093B150026FF0075089505B1EF
:10A1E000038505093B150027FFFF00007510950149
:10A1F000B103093B150026FF0075089503B10385DF
:10A2000006093B150027FFFF000075109501B103FB
:10A21000093B150026FF0075089501B10385070964
:10A220003B150027FFFF000075109501B103093BA6
:10A23000150026FF0075089502B1038508093B1536
:10A240000027FFFF000075109501B103093B1500C1
:10A2500026FF0075089502B1038509093B15002703
:10A26000FFFF000075109501B103093B150026FFA3
:10A270000075089535B103850A093B150027FFFFD6
:10A28000000075109501B103093B150026FF00750C
:10A2900008950CB103850B093B150027FFFF000053
:10A2A00075109501B103093B150026FF007508954F
:10A2B00031B103C0C00403090420034F00630075DB
:10A2C000006C00750073002000560052002C002026
:10A2D0000049006E0063002E0016035400720061F6
:10A2E0000063006B0065007200200044004B00001A
:10A2F0000000000000000000000000000000803F9F
:10A300000000803F0000803F303132333435363733
:10A3100038394142434445464030580030313233A9
:10A3200034353637383961626364656640307800A9
:10A330004C5555555555A53F7751C1166CC156BF63
:10A340009015CB19A001FA3EAD529C804F7E92BE73
:10A35000C4B1B4BD9EEE213ED43888BEE9FAA8BD92
:10A3600000004054FB21F93F3163621A61B4D03DD3
:10A370000000601A61B4D03D7370032E8A19A33BAC
:10A380000000002E8A19A33BC14920259A837B39FE
:10A3900000000000000000006E83F9A22915444E61
:10A3A000D15727FCC0DD34F5999562DB4190433CE1
:10A3B000AB6351FE61C5BBDE3A6E24B7E0D24D42BD
:10A3C000EA2E49061C92D1091CEB1DFE3EA729B1BD
:10A3D000F53582E88444BB2E26709CE9417E5FB44B
:10A3E00039D69139F43953838B5F849C3B28F9BD6E
:10A3F000FF97F81F0F9805DE8B112FEF1F6D0A5A7C
:10A40000CF7E366DB709CB27663F464F2DEA5F9E5C
:10A41000C7BA27757BF1E5EBF739073DEA92528A17
:10A42000B15FFB6B085D8D1FA6F810111111813F04
:10A43000D561C119A0012ABF7DFEB157E31DC73EFA
:10A44000EB9C2B8AE6E55ABE7CD5CF5A3AD9E53D3E
:10A4500002400000000000A00000000005400000D5
:10A46000000000C8000000000C4000000000409CFC
:10A4700000000000194000000020BCBE00000000E9
:10A4800034400000BFC91B8E00000004B54000002E
:10A49000504BCFD06607E2CF010000006C410000B6
:10A4A0003E8251AADFEEA73401000000D94200002D
:10A4B000DCB5A0E23A301F97FFFFFFFFB445000074
:10A4C000FD25A0C8E9A3C14FFFFFFFFFFF3F00002C
:10A4D0000000008000000000FF3F0000000000803E
:10A4E0000000000020A5000800000020000200007D
:10A4F00028010008D0A5000800020020800D0000FF
:10A50000840100081C00000043000000F8FFFFFF6A
:10A510000C0000000E0000000F0000002E000000E4
:10A52000A2012D0102030404200906070809020400
:10A530000608ACA24A041D2919011C141A0353125F
:10A5400054124D1233123212310211301393420C55
:10A5500014080536040A19911C6115020199431B60
:10A5600008BB041387441B089D041ACF04138145BC
:10A570001B08DD041AA1041AAF041ABD04413240BD
:10A58000293C1A6F240916581A7F1C13D2A03308CD
:10A59000121AE40832221B06A14822011AF61029D9
:10A5A000ED13B5A23308041AB90832201AD90832BB
:10A5B00016224C73201A192F01578B803F04E12576
:10A5C000E17A0443EBC84124C3E803F2FFE9102118
:04000005080000ED02
:00000001FF
